:020000040800F2
:1000000000000824CD130008F10F0008F30F0008CA
:10001000F50F0008F70F0008F90F000800000000B6
:10002000000000000000000000000000FB0F0008BE
:10003000FD0F000800000000FF0F0008011000087D
:100040001D1400081D1400081D1400081D140008CC
:100050001D1400081D1400081D14000809100008D4
:100060001D1400081D140008151000082D100008AC
:100070001D1400081D1400081D1400081D1400089C
:100080001D1400081D1400081D1400081D1400088C
:100090001D1400081D1400081D1400081D1400087C
:1000A0001D1400081D1400081D1400081D1400086C
:1000B0003D1000081D1400081D1400081D14000840
:1000C0001D1400081D1400081D1400081D1400084C
:1000D0001D1400084D1000081D1400081D14000810
:1000E0001D1400081D140008000000001D14000865
:1000F0001D1400081D1400081D1400081D1400081C
:100100001D1400081D1400081D1400081D1400080B
:100110001D1400081D1400081D1400081D140008FB
:100120001D1400081D1400081D1400081D140008EB
:100130001D1400081D1400081D1400081D140008DB
:1001400000000000000000000000000000000000AF
:100150001D1400081D1400081D1400081D140008BB
:100160001D1400081D1400085D1000086D10000823
:100170001D1400087D1000081D1400081D1400083F
:100180001D1400081D1400081D1400081D1400088B
:100190001D1400081D1400081D1400081D1400087B
:1001A0001D1400081D1400081D1400081D1400086B
:1001B0001D1400081D1400081D1400081D1400085B
:1001C0001D1400081D1400081D1400081D1400084B
:1001D0001D1400081D1400081D1400081D1400083B
:1001E0001D1400081D1400081D1400081D1400082B
:1001F0001D1400081D1400081D1400081D1400081B
:100200001D1400081D1400081D1400081D1400080A
:100210001D1400081D1400081D1400081D140008FA
:100220001D1400081D1400081D1400080000000023
:100230001D1400081D140008000000001D14000813
:100240001D1400081D1400081D1400081D140008CA
:100250001D1400081D1400081D1400081D140008BA
:100260001D1400081D1400081D1400081D140008AA
:100270001D1400081D1400081D14000800000000D3
:100280001D1400081D1400081D14000800000000C3
:08029000000000001D1400082D
:1002980010B5054C237833B9044B13B10448AFF3B8
:1002A80000800123237010BD3C09002400000000D9
:1002B800689E000808B5034B1BB103490348AFF318
:1002C800008008BD0000000040090024689E000866
:1002D80080F0004002E000BF81F0004142001FBFF3
:1002E8005FEA410392EA030F7FEA226C7FEA236CFC
:1002F8006AD04FEA1262D2EB1363C1BFD2184140F1
:1003080048404140B8BF5B42192B88BF704710F086
:10031800004F40F4000020F07F4018BF404211F029
:10032800004F41F4000121F07F4118BF494292EA91
:10033800030F3FD0A2F1010241FA03FC10EB0C00BD
:10034800C3F1200301FA03F100F0004302D549424A
:1003580060EB4000B0F5000F13D3B0F1807F06D3F7
:1003680040084FEA310102F10102FE2A51D2B1F1EF
:10037800004F40EBC25008BF20F0010040EA0300E4
:100388007047490040EB0000013A28BFB0F5000F64
:10039800EDD2B0FA80FCACF1080CB2EB0C0200FA1A
:1003A8000CF0AABF00EBC25052421843BCBFD04069
:1003B8001843704792F0000F81F4000106BF80F4E3
:1003C80000000132013BB5E74FEA41037FEA226CA6
:1003D80018BF7FEA236C21D092EA030F04D092F071
:1003E800000F08BF0846704790EA010F1CBF0020A5
:1003F800704712F07F4F04D1400028BF40F0004002
:10040800704712F100723CBF00F50000704700F021
:10041800004343F0FE4040F4000070477FEA226248
:1004280016BF08467FEA23630146420206BF5FEA19
:10043800412390EA010F40F4800070474FF0000319
:1004480004E000BF10F0004348BF40425FEA000CE0
:1004580008BF704743F0964301464FF000001CE088
:1004680050EA010208BF70474FF000030AE000BFDE
:1004780050EA010208BF704711F0004302D540421C
:1004880061EB41015FEA010C02BF8446014600208E
:1004980043F0B64308BFA3F18053A3F50003BCFAA9
:1004A8008CF2083AA3EBC25310DB01FA02FC634456
:1004B80000FA02FCC2F12002BCF1004F20FA02F25D
:1004C80043EB020008BF20F00100704702F1200250
:1004D80001FA02FCC2F1200250EA4C0021FA02F2B1
:1004E80043EB020008BF20EADC7070474FF0FF0CB6
:1004F8001CEAD0521EBF1CEAD15392EA0C0F93EAB1
:100508000C0F6FD01A4480EA010C400218BF5FEA52
:1005180041211ED04FF0006343EA501043EA5111C5
:10052800A0FB01310CF00040B1F5000F3EBF4900BF
:1005380041EAD3715B0040EA010062F17F02FD2AC3
:100548001DD8B3F1004F40EBC25008BF20F00100A6
:10055800704790F0000F0CF0004C08BF49024CEABD
:10056800502040EA51207F3AC2BFD2F1FF0340EA4F
:10057800C250704740F400004FF00003013A5DDCC0
:1005880012F1190FDCBF00F000407047C2F1000201
:10059800410021FA02F1C2F1200200FA02FC5FEAEE
:1005A800310040F1000053EA4C0308BF20EADC7038
:1005B800704792F0000F00F0004C02BF400010F4AA
:1005C800000F013AF9D040EA0C0093F0000F01F057
:1005D800004C02BF490011F4000F013BF9D041EA79
:1005E8000C018FE70CEAD15392EA0C0F18BF93EA7B
:1005F8000C0F0AD030F0004C18BF31F0004CD8D1A5
:1006080080EA010000F00040704790F0000F17BF2B
:1006180090F0004F084691F0000F91F0004F14D071
:1006280092EA0C0F01D142020FD193EA0C0F03D1C9
:100638004B0218BF084608D180EA010000F00040CC
:1006480040F0FE4040F40000704740F0FE4040F4A7
:10065800400070474FF0FF0C1CEAD0521EBF1CEA46
:10066800D15392EA0C0F93EA0C0F69D0A2EB030264
:1006780080EA010C49024FEA402037D04FF08053FE
:1006880043EA111143EA10130CF000408B4238BFC3
:100698005B0042F17D024FF4000C8B4224BF5B1AD1
:1006A80040EA0C00B3EB510F24BFA3EB510340EA1F
:1006B8005C00B3EB910F24BFA3EB910340EA9C00CD
:1006C800B3EBD10F24BFA3EBD10340EADC001B013D
:1006D80018BF5FEA1C1CE0D1FD2A3FF650AF8B42E1
:1006E80040EBC25008BF20F0010070470CF0004CEE
:1006F8004CEA50207F32C2BFD2F1FF0340EAC25019
:10070800704740F400004FF00003013A37E792F0D9
:10071800000F00F0004C02BF400010F4000F013A37
:10072800F9D040EA0C0093F0000F01F0004C02BF32
:10073800490011F4000F013BF9D041EA0C0195E79B
:100748000CEAD15392EA0C0F08D142027FF47DAF34
:1007580093EA0C0F7FF470AF084676E793EA0C0F24
:1007680004D14B023FF44CAF08466EE730F0004C22
:1007780018BF31F0004CCAD130F000427FF45CAFB2
:1007880031F000437FF43CAF5FE700BF42000ED278
:10079800B2F1FE4F0BD34FF09E03B3EB126209D4B4
:1007A8004FEA002343F0004323FA02F070474FF06A
:1007B8000000704712F1610F01D1420202D14FF0DF
:1007C800FF3070474FF00000704700BF53B94AB977
:1007D800002908BF00281CBF4FF0FF314FF0FF3041
:1007E80000F074B9ADF1080C6DE904CE00F006F81C
:1007F800DDF804E0DDE9022304B070472DE9F04795
:10080800089E0D4604468846002B4DD18A429446E0
:1008180068D9B2FA82F252B101FA02F3C2F12001A8
:1008280020FA01F10CFA02FC41EA030894404FEA6D
:100838001C45210CB8FBF5FE1FFA8CF705FB1E833F
:1008480041EA03430EFB07F199420BD91CEB030362
:100858000EF1FF3080F01E81994240F21B81AEF10B
:10086800020E63445B1AA4B2B3FBF5F005FB103328
:1008780044EA034400FB07F7A7420AD91CEB040427
:1008880000F1FF3380F00881A74240F205816444FB
:100898000238E41B40EA0E4000211EB1D440002378
:1008A800C6E90043BDE8F0878B4208D9002E00F066
:1008B800EE800021C6E900050846BDE8F087B3FAD6
:1008C80083F100294AD1AB4202D3824200F2F98077
:1008D800841A65EB030301209846002EE2D0C6E98E
:1008E8000048DFE702B9FFDEB2FA82F2002A40F0E0
:1008F8009180A1EB0C054FEA1C471FFA8CFE0121E1
:10090800B5FBF7F307FB1350250C45EA00450EFB32
:1009180003F0A84208D91CEB050503F1FF3802D201
:10092800A84200F2CB8043462D1AA4B2B5FBF7F0DB
:1009380007FB105544EA05440EFB00FEA64508D9FE
:100948001CEB040400F1FF3502D2A64500F2BB807F
:100958002846A4EB0E0440EA03409EE7C1F12007B5
:100968008B4022FA07FC4CEA030C20FA07F405FA3C
:1009780001F31C43FD404FEA1C4900FA01F3B5FBA3
:10098800F9F8200C1FFA8CFE09FB185540EA0545BA
:1009980008FB0EF0A84202FA01F20BD91CEB050580
:1009A80008F1FF3A80F08880A84240F28580A8F1DB
:1009B800020865442D1AA4B2B5FBF9F009FB1055DD
:1009C80044EA054500FB0EFEAE4508D91CEB0505BB
:1009D80000F1FF346CD2AE456AD90238654440EA6A
:1009E8000840A0FB0294A5EB0E05A542C846A64602
:1009F80056D353D05EB1B3EB080265EB0E0505FA8A
:100A080007F722FA01F3CD401F43C6E9007500211C
:100A1800BDE8F087C2F1200320FA03F10CFA02FCCA
:100A280025FA03F395400D434FEA1C471FFA8CFE45
:100A3800B3FBF7F107FB11302B0C43EA004301FB32
:100A48000EF0984204FA02F408D91CEB030301F1F2
:100A5800FF382FD298422DD9023963441B1AADB200
:100A6800B3FBF7F007FB103345EA034500FB0EF331
:100A7800AB4208D91CEB050500F1FF3816D2AB4292
:100A880014D902386544ED1A40EA014138E7314685
:100A9800304607E78646E5E61846FAE64B45A9D20A
:100AA800B9EB020864EB0C0E0138A3E74046EAE70D
:100AB800204694E74146D1E7D0467BE7023B6544B0
:100AC80032E7084609E76444023842E7704700BF46
:100AD80000B583B00B4BD3F8D82042F00102C3F81D
:100AE800D820D3F8D83003F001030193019B0022EA
:100AF80011460B2000F024FD0B2000F057FD03B039
:100B08005DF804FB0044025830B58BB0002405940E
:100B18000694079408940994294BD3F8E02042F0EE
:100B28008002C3F8E020D3F8E02002F080020192AE
:100B3800019AD3F8E02042F00402C3F8E020D3F889
:100B4800E02002F004020292029AD3F8E02042F078
:100B58000102C3F8E020D3F8E02002F0010203927A
:100B6800039AD3F8E02042F00202C3F8E020D3F859
:100B7800E03003F002030493049B022305934FF42F
:100B88008815069505A90F4801F00EFF1023059357
:100B98000695079405A90C4801F006FF2246214650
:100BA800072000F0CDFC072000F000FD224621467A
:100BB8000A2000F0C5FC0A2000F0F8FC0BB030BD9C
:100BC800004402580008025800000258022800D0C9
:100BD8007047084B1B78002BFAD110B5064C2360E0
:100BE80000F07CFC2060082000F0EEFC014B0122A4
:100BF8001A7010BD580900246009002410B584B08B
:100C08000024009401940294039400F003FD01234E
:100C18008DF800308DF801404FF0105201921222E9
:100C28008DF808208DF809408DF80A4003228DF8C8
:100C38000B208DF80C408DF80D308DF80E308DF8A6
:100C48000F40684600F004FD042000F0F1FC04B0F9
:100C580010BD000010B4164B1A68164B1A54411CEC
:100C6800C2F307245C54811CC2F307445C54C11CC2
:100C7800120E5A54104A1468011D5C541168090A6E
:100C880000F1050C03F80C101168090C00F1060CB2
:100C980003F80C101268120EC11D5A5400F1080214
:100CA8000D2199540930FF221A5410BC704700BF17
:100CB8004C0D0024640900245C09002472B6FEE788
:100CC80000B59FB04C2200210BA808F03FF8202265
:100CD800002103A808F03AF8022002F0F5FD0023ED
:100CE8000093394BDA6A22F00102DA62DB6A03F018
:100CF80001030093354B9A6942F440429A619B691B
:100D080003F440430093009B304B9B6913F4005F4E
:100D1800FAD02F4BD3F8F42042F00202C3F8F420A3
:100D2800D3F8F43003F002030193019B00230293EC
:100D3800264B9A6942F440429A619B6903F4404306
:100D48000293214BDA6A42F00102DA62DB6A03F0AD
:100D580001030293029B1D4B9B6913F4005FFAD0B9
:100D680021230B934FF480330C9301231193022317
:100D7800149315931693F0221792189319931A93B4
:100D880008231B9300231C931D930BA802F0CEFD90
:100D9800B0B93F2303930323049300230593082347
:100DA80006934023079308934FF4806209920A93AD
:100DB800042103A803F020FA20B91FB05DF804FB52
:100DC800FFF77CFFFFF77AFF00040058004802583D
:100DD8000044025810B5FFF711FF404B5B6913F44C
:100DE800003F13D1BFF34F8FBFF36F8F3B4B0022F0
:100DF800C3F85022BFF34F8FBFF36F8F5A6942F485
:100E080000325A61BFF34F8FBFF36F8F334B5B696B
:100E180013F4803F27D1314B0022C3F88420BFF35D
:100E28004F8FD3F88000C0F34E3200E01A46C0F36B
:100E3800C90143F6E07303EA421343EA8173274C7E
:100E4800C4F860320B460139002BF2D1531E002A38
:100E5800ECD1BFF34F8F636943F480336361BFF311
:100E68004F8FBFF36F8F00F0FFFAFFF729FFFFF7EF
:100E78004BFEFFF72DFE00F087F900F0F7F907F0B9
:100E880079FC174800F03AF83C21164804F095FD23
:100E980021E0426A144B1A60134B1B689942F8D040
:100EA80000F01CFB114B1B68C01A114B1860204640
:100EB800FFF7D0FE0A34B4F57A7F07DA094B1868D1
:100EC800416A0C4B1960084B1960E5E74FF47A71D9
:100ED800094807F0A3FC0024EDE700BF00ED00E09F
:100EE800200E00245C0D00244C0D00246009002411
:100EF8005C090024500D00246409002408B5054B42
:100F08001860054B1868002302221946806807F00C
:100F18006FFF08BD540D0024FC00002410B50138F3
:100F280001280AD814464FF0FF3392B207480068E8
:100F380005F0D8FB40B9204610BD07F0DDFE0923B7
:100F480003604FF0FF30F7E70520F5E7540D002464
:100F5800022801D80020704708B507F0CDFE092304
:100F680003604FF0FF3008BD08B507F0C5FE092340
:100F780003604FF0FF3008BD08B548B94FF0FF33A4
:100F880001220848006805F015FC40B9012008BD99
:100F980007F0B2FE092303604FF0FF30F7E70520A2
:100FA800F5E700BF540D002408B5022804D84FF413
:100FB80000534B60002008BD07F09EFE0923036024
:100FC800F8E7000082B0074BD3F8F42042F00202A1
:100FD800C3F8F420D3F8F43003F002030193019B23
:100FE80002B0704700440258FEE7FEE7FEE7FEE75E
:100FF800FEE770477047704708B500F063FA08BD10
:1010080008B5022001F0E4FD08BD000008B5102075
:1010180001F0DEFD024B1B6800225A6208BD00BFCA
:101028005C0D002408B5024801F022F908BD00BF94
:10103800A80D002408B5024804F00BFB08BD00BF4A
:101048005C0D002408B5024804F0BCFD08BD00BFD3
:10105800200E002408B5024802F0F7F808BD00BFCA
:101068009823002408B5024802F0EFF808BD00BF35
:101078009823002408B5024802F0E7F808BD00BF2D
:101088009823002410B503460C4A0D490D48006802
:1010980040B10C4800680344521A934206D8094AE2
:1010A800136010BD0748084C0460F2E707F024FEFF
:1010B8000C2303604FF0FF30F3E700BF0000082463
:1010C80000040000580D0024E82A0024244B1B6863
:1010D80003F00F03062B06D8214A136823F00F03E9
:1010E80043F0070313601F4B1A6842F001021A60AD
:1010F80000221A6119681C4A0A401A60184B1B68BA
:1011080013F0080F06D0164A136823F00F0343F0B4
:1011180007031360134B00229A61DA611A621349BC
:1011280099621349D962134919635A639963DA6357
:1011380019645A64196821F4802119601A660E4BE3
:101148001A680E4B1340B3F1005F03D20C4B012217
:10115800C3F808210B4B43F2D2021A60704700BF54
:1011680000200052004402587FEDF6EA0002020215
:101178000000FF01800201010010005C0000FFFF79
:10118800008000510040005200B58DB0242200219B
:1011980003A807F0DBFD0023009301930293124894
:1011A8004FF0804202600322426083604FF0FF31BB
:1011B800C16003618361039201230593099303A925
:1011C80004F08EFB50B90023009302936946064849
:1011D80004F058FC28B90DB05DF804FBFFF76EFD6C
:1011E800F1E7FFF76BFDF6E75C0D002400B589B069
:1011F8000023039304930593069307930368B3F1BD
:10120800804F02D009B05DF804FB164BD3F8E820F4
:1012180042F00102C3F8E820D3F8E82002F0010206
:101228000192019AD3F8E02042F00102C3F8E020CD
:10123800D3F8E03003F001030293029B03230393E6
:10124800022304930123079303A9074801F0ACFB89
:10125800002211461C2000F073F91C2000F0A6F9AA
:10126800D0E700BF004402580000025808B51748EC
:10127800174B03604FF4E133436000238360C3607E
:1012880003610C2242618361C3610362436283622A
:1012980005F080FB70B900210C4805F0F7FB60B938
:1012A80000210A4805F017FC50B9084805F0CFFBA3
:1012B80048B908BDFFF702FDEDE7FFF7FFFCEFE7D0
:1012C800FFF7FCFCF1E7FFF7F9FCF2E7200E00243A
:1012D8000010014030B5B9B0044600213391349173
:1012E800359136913791C02202A807F02FFD226868
:1012F8002F4B9A4201D039B030BD01220023CDE9ED
:10130800022302A803F014FA00284AD1294BD3F883
:10131800F02042F01002C3F8F020D3F8F02002F0D9
:1013280010020092009AD3F8E02042F00102C3F8BC
:10133800E020D3F8E03003F001030193019B4FF460
:10134800C0633393022334930025359536950723DC
:10135800379333A9184801F027FB1848184B036046
:101368002A23436040238360C5604FF48063036190
:10137800456185614FF48073C3610562456200F081
:10138800CDFA88B90D4BE3679C63002211462520EE
:1013980000F0D6F8252000F009F9E06F00F0BEFA59
:1013A800A9E7FFF78BFCB1E7FFF788FCEAE700BF86
:1013B800001001400044025800000258A80D002403
:1013C80010000240DFF834D0FFF780FE0C480D49CA
:1013D8000D4A002302E0D458C4500433C4188C4288
:1013E800F9D30A4A0A4C002301E013600432A242EE
:1013F800FBD307F087FCFFF7EDFC704700000824DB
:10140800000000243C090024209F00083C09002417
:10141800E42A0024FEE70000104B1B780BB90120DA
:10142800704710B504464FF47A70B0FBF3F30C4ADA
:101438001068B0FBF3F000F0D9F868B90F2C01D9A7
:1014480001200AE0002221464FF0FF3000F078F832
:10145800044B1C60002000E0012010BD080000249F
:10146800000000240C00002410B5032000F056F8FA
:1014780002F0B6FD0F498B69C3F303230E4AD35C10
:1014880003F01F03D8408B6903F00F03D35C03F00C
:101498001F0320FA03F3094A1360094B18600F2051
:1014A800FFF7BAFF10B10124204610BD0446FFF72C
:1014B80089FDF9E700440258809E000804000024D2
:1014C80000000024034B1B78034A11680B44136087
:1014D800704700BF08000024B40E0024014B1868B0
:1014E800704700BFB40E002438B50446FFF7F6FF76
:1014F8000546B4F1FF3F02D0044B1B781C44FFF7AC
:10150800EDFF401BA042FAD338BD00BF08000024FD
:10151800014B1868000C70470010005C0649CB6846
:1015280023F4E0631B041B0C000200F4E060034397
:10153800024A1A43CA60704700ED00E00000FA054D
:1015480000B5174BDB68C3F30223C3F1070CBCF1EA
:10155800040F28BF4FF0040C03F1040EBEF1060F70
:1015680014D9033B4FF0FF3E0EFA0CFC21EA0C01A4
:1015780099400EFA03F322EA03031943002807DB14
:101588000901C9B2074B19545DF804FB0023E9E7C8
:1015980000F00F000901C9B2034B1954F4E700BF6A
:1015A80000ED00E000E400E014ED00E0002807DBB7
:1015B80000F01F02400901239340024A42F82030FC
:1015C800704700BF00E100E000280CDB00F01F02BC
:1015D8004009012393402030034A42F82030BFF3EA
:1015E8004F8FBFF36F8F704700E100E00138B0F113
:1015F800807F0BD24FF0E0235861054AF02182F832
:1016080023100020986107221A6170470120704753
:1016180000ED00E0BFF35F8F044B5A6A22F480327A
:101628005A620022C3F89420704700BF00ED00E022
:1016380040F00100054BC3F894005A6A42F4803226
:101648005A62BFF34F8FBFF36F8F704700ED00E012
:101658004378144AC2F89830D2F8A03023F0010336
:10166800C2F8A0304368C2F89C30017BC37A1B06DD
:1016780043EA0173817A43EAC143417B43EA8143E8
:10168800817B43EA4143C17B43EA0143417A43EA10
:101698000123017A43EA410301780B43C2F8A030E1
:1016A800704700BF00ED00E003682749274A9342CE
:1016B80018BF8B422FD0183293422CD01832934245
:1016C80029D01832934226D01832934223D01832A8
:1016D800934220D0183293421DD002F5567293429D
:1016E80019D01832934216D01832934213D01832B8
:1016F800934210D0183293420DD0183293420AD038
:101708001832934207D01832934204D023F0FF03D3
:101718008365806D704710B4D9B210390C4AA2FBAA
:101728000142C2F302120B4CA25CC2655F2906D9C2
:10173800094A1A4004328265806D10BC7047064A17
:101748001A408265F8E700BF1000024028000240F6
:10175800ABAAAAAA909E000800FCFFFF83699BB968
:10176800836A012B0AD0022B02D00BB100207047EC
:10177800C36A13F0807F2AD100207047C36AB3F18F
:10178800C07F26D000207047B3F5005F0AD0836A77
:10179800022B26D9032B26D1C36A13F0807F24D1CC
:1017A80000207047836A032B03D8DFE803F0140492
:1017B800140A00207047C36A13F0807F0DD10020FF
:1017C8007047C36AB3F1C07F09D000207047012079
:1017D80070470120704701207047012070470120A1
:1017E80070470120704700207047012070470000B3
:1017F80003682249224A934218BF8B4228D01432E8
:10180800934225D01432934222D0143293421FD0EF
:10181800143293421CD01432934219D0143293429A
:1018280016D0DAB2103A1749A1FB0212120916496A
:101838001944A8291FD9154B13449B000366144B60
:10184800436602F01F02012303FA02F28266704720
:10185800DBB2083B0F4AA2FB03230F4A02EB131229
:10186800920002660D4A4266C3F30413012202FA8B
:1018780003F3836670470832DDE700BF0854025857
:101888001C540258ABAAAAAAF0FBFDBF00820010A4
:1018980080080240CDCCCCCC009600168058025867
:1018A80001794A1E072A2CD830B40368154D164C06
:1018B800A34218BFAB4218D01434A34215D0143435
:1018C800A34212D01434A3420FD01434A3420CD034
:1018D8001434A34209D01434A34206D00B4B0B4452
:1018E8009B00C3660A4B036705E00A4B0B449B0049
:1018F800C366094B0367012303FA02F2426730BC4F
:1019080070477047085402581C5402583F82001010
:10191800400902403F9600164059025870B50446E7
:10192800FFF7DCFD002C00F0B6810546236853491B
:10193800534A934218BF8B420CBF0122002250D059
:1019480030318B424DD018318B424AD018318B42FE
:1019580047D018318B4244D018318B4241D01831CE
:101968008B423ED001F556718B423AD018318B42EA
:1019780037D018318B4234D018318B4231D01831DE
:101988008B422ED018318B422BD018318B4228D065
:1019980018318B4225D03B493B4A934218BF8B42B2
:1019A80000F03181394A934200F02D81143293427C
:1019B80000F029811432934200F0258114329342B9
:1019C80000F021811432934200F01D8114329342B9
:1019D80000F0198140236365032384F83530012022
:1019E8004AE0022184F83510002184F834107ABBCB
:1019F800274A93422CD01832934229D01832934266
:101A080026D01832934223D01832934220D018326D
:101A180093421DD002F55672934219D01832934260
:101A280016D01832934213D01832934210D018327D
:101A380093420DD0183293420AD01832934207D0FD
:101A48001832934204D01A6822F001021A6003E0A7
:101A58001A6822F001021A6023681A6812F0010F4E
:101A680018D0FFF73BFD431B052BF5D920236365F1
:101A7800032384F83530012070BD00BF10000240F8
:101A880028000240085402581C5402583054025886
:101A9800400002401A6881481040A168E2680A4381
:101AA80021690A4361690A43A1690A43E1690A4352
:101AB800216A0A430243616A042900F0998078493F
:101AC800086878490140B1F1005F11D36168A1F15C
:101AD8002905A1F13F00032888BF052D06D9A1F1EA
:101AE8004700012802D94F39032901D842F480124E
:101AF8001A602668756925F00705636A1D43042B7B
:101B080008D1A36A1D43E36A23B12046FFF726FEE6
:101B1800002872D175612046FFF7C6FDE36D03F01A
:101B28001F023F239340836023685F495F4A9342C3
:101B380018BF8B4242D0183293423FD0183293429A
:101B48003CD01832934239D01832934236D01832EA
:101B5800934233D01832934230D002F556729342F2
:101B68002CD01832934229D01832934226D01832FA
:101B7800934223D01832934220D0183293421DD07A
:101B8800183293421AD01832934217D0484A9342D7
:101B980014D01432934211D0143293420ED014321E
:101BA80093420BD01432934208D01432934205D09A
:101BB8001432934202D01432934213D12046FFF7D5
:101BC80017FEA368802B59D0236E22791A60636EA2
:101BD800A26E5A606368013B072B52D90023E36663
:101BE8002367636700206065012384F8353043E785
:101BF800E16A206B01430A4361E7402363650120E2
:101C080084F8350038E7022284F83520002284F869
:101C180034201A6827491140A268402A2CD0802A0B
:101C280027D00022E06842EAD002206942EAD002C6
:101C3800606942EAD002A06942EAD002E06942EA59
:101C4800D002206A42EA10120A431A6022681A4B2C
:101C580013441A4AA2FB03231B099B00E365204691
:101C6800FFF722FDE26D02F01F0101228A40426067
:101C78005AE74FF48042D5E71022D3E70023636088
:101C8800A2E72046FFF70CFEE36E00221A60236FDE
:101C9800626F5A60A6E70120EEE600BF3F8010FEA3
:101CA8000010005C0000FFFF100002402800024006
:101CB800085402580F00FEFFF8ABFDA7CDCCCCCCE2
:101CC80070B50446FFF70AFC002C00F09181054628
:101CD80094F83530DBB2022B06D0802363650023ED
:101CE80084F83430012070BD23688C498C4A9342B3
:101CF80018BF8B4230D0183293422DD018329342FD
:101D08002AD01832934227D01832934224D018325E
:101D1800934221D0183293421ED002F55672934254
:101D28001AD01832934217D01832934214D018326E
:101D3800934211D0183293420ED0183293420BD0EE
:101D48001832934208D01832934205D01A6822F00C
:101D58000E021A60266809E01A6822F01E021A604C
:101D68002268536923F080035361266823686B490E
:101D78006B4A934218BF8B4242D0183293423FD0ED
:101D8800183293423CD01832934239D018329342D9
:101D980036D01832934233D01832934230D002F5FD
:101DA800567293422CD01832934229D0183293425B
:101DB80026D01832934223D01832934220D01832BA
:101DC80093421DD0183293421AD01832934217D03A
:101DD800544A934214D01432934211D0143293428D
:101DE8000ED0143293420BD01432934208D01432DE
:101DF800934205D01432934202D01432934204D154
:101E0800226E136823F48073136023684349444A9D
:101E1800934218BF8B422FD0183293422CD01832DD
:101E2800934229D01832934226D01832934223D0B5
:101E38001832934220D0183293421DD002F55672C0
:101E4800934219D01832934216D01832934213D0C5
:101E58001832934210D0183293420DD01832934260
:101E68000AD01832934207D01832934204D01A6825
:101E780022F001021A6003E01A6822F001021A60D7
:101E8800336813F0010F0ED0FFF728FB431B052B17
:101E9800F6D920236365032384F83530002384F8BA
:101EA800343001201FE723681C491D4A934218BF9C
:101EB8008B4239D01832934236D01832934233D0FD
:101EC8001832934230D0183293422DD018329342B0
:101ED8002AD01832934227D002F55672934223D063
:101EE8001832934220D0183293421DD018329342B0
:101EF8001AD01832934217D01832934214D018329D
:101F0800934211D0183293420ED0A16DE36D03F0C5
:101F18001F02012393404B600DE000BF10000240F8
:101F28002800024008540258A16DE36D03F01F0217
:101F38003F2393408B6023682E492F4A934218BF52
:101F48008B4242D0183293423FD0183293423CD051
:101F58001832934239D01832934236D0183293420D
:101F680033D01832934230D002F5567293422CD0B7
:101F78001832934229D01832934226D0183293420D
:101F880023D01832934220D0183293421DD01832F1
:101F980093421AD01832934217D0184A934214D059
:101FA8001432934211D0143293420ED01432934219
:101FB8000BD01432934208D01432934205D0143215
:101FC800934202D0143293420BD1636EA26E5A60D0
:101FD800E36E33B11A6822F480721A60236F626F5D
:101FE8005A60012384F83530002084F834007AE6FA
:101FF800012078E6100002402800024008540258E8
:10200800002800F0298108B5024690F83530DBB287
:10201800022B03D080234365012008BD0368904844
:1020280090498B4218BF83420CBF0121002166D022
:102038003030834263D01830834260D018308342F6
:102048005DD0183083425AD01830834257D01830A8
:10205800834254D000F55670834250D018308342E2
:102068004DD0183083424AD01830834247D01830B8
:10207800834244D01830834241D0183083423ED046
:10208800183083423BD0196821F00E01196013689B
:10209800A0F5956073498B4218BF83426AD0724994
:1020A8008B4267D018318B4264D018318B4261D093
:1020B80018318B425ED018318B425BD018318B427D
:1020C80058D001F556718B4254D018318B4251D0FB
:1020D80018318B424ED018318B424BD018318B427D
:1020E80048D018318B4245D018318B4242D0183134
:1020F8008B423FD0196821F0010119603EE00420AD
:1021080082F8350081BB584A93422DD01832934249
:102118002AD01832934227D01832934224D018324A
:10212800934221D0183293421ED002F55672934240
:102138001AD01832934217D01832934214D018325A
:10214800934211D0183293420ED0183293420BD0DA
:102158001832934208D01832934205D01A6822F0F8
:1021680001021A60002058E71A6822F001021A607A
:10217800002052E7196821F00101196013683848F6
:1021880038498B4218BF834242D018318B423FD026
:1021980018318B423CD018318B4239D018318B42E0
:1021A80036D018318B4233D018318B4230D001F5FC
:1021B80056718B422CD018318B4229D018318B4262
:1021C80026D018318B4223D018318B4220D01831B9
:1021D8008B421DD018318B421AD018318B4217D040
:1021E80022498B4214D014318B4211D014318B42C6
:1021F8000ED014318B420BD014318B4208D01431DD
:102208008B4205D014318B4202D014318B4217D146
:10221800116E0B6823F480730B60906DD36D03F01F
:102228001F0101238B404360536E916E5960D36E3A
:1022380033B1196821F480711960136F516F5960B7
:10224800012382F83530002382F83430136D2BB126
:10225800104698470020E0E6012070470020DCE6A1
:102268001000024028000240400002400854025872
:10227800F0B583B00446002301937D4B1D687D4B68
:10228800A3FB0535AD0A876D3E68D7F800C0036823
:1022980079497A48834218BF8B420CBF012000203D
:1022A80061D0774A93425ED0183293425BD018329D
:1022B800934258D01832934255D01832934252D094
:1022C800183293424FD002F5567293424BD01832CF
:1022D800934248D01832934245D01832934242D0A4
:1022E800183293423FD0183293423CD0183293426E
:1022F80039D01832934236D06249634A934218BFA4
:102308008B4212D0614A93420FD0143293420CD0C0
:102318001432934209D01432934206D014329342B5
:1023280003D01432934240F061821A68E16D01F0E3
:102338001F010420884010EA0C0F00F0A78212F059
:10234800040F00F0A382786012F4004F00F05A8264
:1023580012F4803F40F05082A36C002B00F04682BC
:102368002046984742E2E26D02F01F0108228A40A7
:10237800324241D070BB424A93422BD0183293422A
:1023880028D01832934225D01832934222D01832DE
:1023980093421FD0183293421CD002F556729342D2
:1023A80018D01832934215D01832934212D01832EE
:1023B80093420FD0183293420CD01832934209D06E
:1023C8001832934206D01832934203D01A68C2F3E7
:1023D800C00202E01A68C2F380026AB11A6822F0E9
:1023E80004021A60E36D03F01F0208239340BB60E8
:1023F800636D43F001036365E26D02F01F0226FA84
:1024080002F313F0010F47D023681B481B498B4286
:1024180018BF83423CD018318B4239D018318B42D7
:1024280036D018318B4233D018318B4230D0183126
:102438008B422DD018318B422AD001F556718B4230
:1024480026D018318B4223D018318B4220D0183136
:102458008B421DD018318B421AD018318B4217D0BD
:1024680018318B4214D018318B4211D01B6813E0FD
:1024780000000024B5814E1B1000024028000240D5
:1024880040000240085402581C5402583054025864
:102498005B6913F0800F3BD1E36D03F01F03042247
:1024A80002FA03F3334240D02268964896498A429A
:1024B80018BF824235D018318A4232D018318A4248
:1024C8002FD018318A422CD018318A4229D018319D
:1024D8008A4226D018318A4223D001F556718A42A1
:1024E8001FD018318A421CD018318A4219D01831AD
:1024F8008A4216D018318A4213D018318A4210D035
:1025080018318A420DD018318A420AD013680CE07B
:10251800012303FA02F2BA60636D43F002036365B4
:10252800BAE7126812F0020F3DD1E36D03F01F0302
:10253800102202FA03F333425FD0226871487249CD
:102548008A4218BF824234D018318A4231D01831B9
:102558008A422ED018318A422BD018318A4228D08C
:1025680018318A4225D018318A4222D001F5567195
:102578008A421ED018318A421BD018318A4218D09C
:1025880018318A4215D018318A4212D018318A423D
:102598000FD018318A420CD018318A4209D01268FB
:1025A800C2F3800208E0BB60636D43F00403636517
:1025B800BBE71268C2F3C002FAB1BB6023681A68AD
:1025C80012F4802F0DD01B6813F4002F04D1236C54
:1025D8009BB12046984710E0A36C73B120469847FA
:1025E8000BE01A6812F4807F03D11A6822F00802FF
:1025F8001A60236C0BB120469847E36D03F01F0364
:10260800202202FA03F3334200F0928022683D4808
:102618003D498A4218BF82422ED018318A422BD0B7
:1026280018318A4228D018318A4225D018318A4276
:1026380022D018318A421FD018318A421CD001F5A5
:1026480056718A4218D018318A4215D018318A42F8
:1026580012D018318A420FD018318A420CD0183162
:102668008A4209D018318A4206D018318A4203D0EA
:102678001268C2F3400202E01268C2F30012002A94
:1026880056D0BB6094F83530DBB2042B0ED02368EB
:102698001A6812F4802F39D01B6813F4002F2CD13C
:1026A800636C002B44D02046984741E022681368A9
:1026B80023F0160313602268536923F080035361E3
:1026C800236CB3B12268136823F008031360E36D29
:1026D80003F01F023F239340BB60012384F8353089
:1026E800002384F83430236D002B7FD02046984790
:1026F8007CE0A36C002BE5D1E9E7E36BC3B120468E
:10270800984715E010000240280002401A6812F4A9
:10271800807F09D11A6822F010021A60012384F818
:102728003530002384F83430E36B0BB120469847EA
:10273800636D002B5AD0636D13F0010F52D0042340
:1027480084F8353023689649964A934218BF8B42DD
:102758002FD0183293422CD01832934229D01832F5
:10276800934226D01832934223D01832934220D075
:10277800183293421DD002F55672934219D018327E
:10278800934216D01832934213D01832934210D085
:10279800183293420DD0183293420AD0183293421D
:1027A80007D01832934204D01A6822F001021A6046
:1027B80003E01A6822F001021A60019B01330193B9
:1027C800AB4204D823681B6813F0010FF5D12368C6
:1027D8001B6813F0010F0BD0032384F83530002356
:1027E80084F83430E36C0BB12046984703B0F0BD51
:1027F800012384F83530F2E7236C002BF6D020460D
:102808009847F3E712F0200F3AD123686449654AE4
:10281800934218BF8B422FD0183293422CD01832D3
:10282800934229D01832934226D01832934223D0AB
:102838001832934220D0183293421DD002F55672B6
:10284800934219D01832934216D01832934213D0BB
:102858001832934210D0183293420DD01832934256
:102868000AD01832934207D01832934204D01A681B
:1028780022F004021A6003E01A6822F008021A60C3
:10288800236C002BB2D020469847AFE7022088403F
:1028980010EA0C0F60D012F0020F5DD0786012F4CD
:1028A800004F0ED012F4803F05D1636C002B9DD0F1
:1028B800204698479AE7E36B002B97D02046984725
:1028C80094E712F0200F40D123683549354A9342E6
:1028D80018BF8B422FD0183293422CD01832934213
:1028E80029D01832934226D01832934223D0183276
:1028F800934220D0183293421DD002F5567293426B
:1029080019D01832934216D01832934213D0183285
:10291800934210D0183293420DD0183293420AD005
:102928001832934207D01832934204D01A6822F022
:102938000A021A6003E01A6822F014021A600123DE
:1029480084F83530002384F83430E36B002B3FF4EF
:102958004DAF2046984749E7082000FA01F111EAEF
:102968000C0F3FF443AF12F0080F3FF43FAF1A6863
:1029780022F00E021A60E36D03F01F03012202FA2F
:1029880003F37B60626584F83520002384F83430D3
:10299800E36C002B3FF42AAF2046984726E700BF98
:1029A800100002402800024070B582B000236EE09B
:1029B80085685E000324B44025EA0405CC68B44069
:1029C8002C438460446824EA0C0C4C68C4F300145B
:1029D8009C4044EA0C0444606CE0DD08083550F87B
:1029E800256003F007044FEA840C0F2404FA0CF462
:1029F80026EA040E0C6904FA0CF444EA0E0440F8C2
:102A080025406FE0092400E0002404FA0EF42C436A
:102A18000CF1020C6B4D45F82C404FF0B044256882
:102A2800D44325EA0206D1F804C01CF4801F01D063
:102A380042EA05064FF0B0452E606D6804EA0506C7
:102A4800D1F804C01CF4001F01D042EA05064FF07B
:102A5800B0456E60D5F8845004EA0506D1F804C084
:102A68001CF4003F01D042EA05064FF0B045C5F816
:102A78008460D5F880502C404E6816F4803F01D011
:102A880042EA05044FF0B042C2F8804001330A68B8
:102A980032FA03F400F093804FF0010C0CFA03FCB7
:102AA8001CEA0202F2D04C6804F00304013C012C39
:102AB8007FF67EAF4C6804F00304032C0CD0C46886
:102AC8005D004FF0030C0CFA05FC24EA0C0C8C6832
:102AD800AC4044EA0C04C4604C6804F00304022CC3
:102AE8003FF47BAF04684FEA430E4FF0030C0CFA37
:102AF8000EFC24EA0C0C4C6804F0030404FA0EF4EF
:102B080044EA0C0404604C6814F4403FBED02E4CD8
:102B1800D4F8F45045F00205C4F8F450D4F8F44061
:102B280004F002040194019C4FEA930C0CF1020595
:102B3800244C54F8255003F003044FEA840E0F2464
:102B480004FA0EF425EA0405204CA0423FF45CAFD9
:102B580004F58064A04222D004F58064A04220D00D
:102B680004F58064A0421ED004F58064A0421CD005
:102B780004F58064A0421AD004F58064A04218D0FD
:102B880004F58064A04216D004F58064A04214D0F5
:102B980004F58064A0423FF435AF0A2435E70124E8
:102BA80033E7022431E703242FE704242DE7052423
:102BB8002BE7062429E7072427E7082425E702B09E
:102BC80070BD00BF000400580044025800000258BD
:102BD80008B54FF0B043D3F88830034200D108BDA0
:102BE8004FF0B043C3F88800FDF7F0FFF7E72DE991
:102BF800F04383B0D0F8008001EBC10300EB8303FE
:102C08009A6A5B6A9A4254D807460C469B1A01EBAB
:102C1800C10200EB8202D2699A4200D31A4602F13D
:102C280003094FEA990915E006F103094FEA9909E2
:102C3800BB7904EBC40507EB8505296A0093B3B299
:102C4800E2B2404604F0A4FA2B6A33442B62AB6A22
:102C58003344AB6208EB441303F510639B699BB2E2
:102C68004B4512D304EBC40207EB8202916A536A04
:102C780099420AD24BB15B1A04EBC40207EB8202F9
:102C8800D6699E42D0D31E46CEE704EBC40007EBBC
:102C980080077A6ABB6A9A420FD804F00F040123AE
:102CA800A340D8F8344824EA0304C8F8344800207C
:102CB80000E0012003B0BDE8F0830020FAE730B55A
:102CC80083B000287AD0044690F89534ABB103233A
:102CD80084F89534206804F013F8237C8DF80030CC
:102CE800231D0ECB206803F041FF58B1022384F85E
:102CF80095340125284603B030BD80F8943405F09A
:102D08003DFEE4E70021206804F05DFC024608B9B6
:102D1800034617E0022384F895340125EAE703EB1C
:102D2800C30104EB8101012048750B75CB85002098
:102D38000876C861086203EBC30104EB81014862AD
:102D48000133DBB220799842E9D816E002EBC203DE
:102D580004EB8303002183F8551283F8542283F887
:102D68005812C3F85C12C3F8601202EBC20304EBFA
:102D78008303C3F864120132D2B29042E6D8237CAE
:102D88008DF80030231D0ECB206804F00FF805469F
:102D980058B900236374012384F89534237B012BED
:102DA80008D0206804F0CDFBA4E7022384F895340A
:102DB80001259FE7204600F071FDF2E7012599E71C
:102DC800036890F89424012A1AD010B50446012209
:102DD80080F89424DA6812F0400F02D0427B012A6E
:102DE80009D0206803F086FF206804F09CFB0020CF
:102DF80084F8940410BD9A6B42F480329A63F0E729
:102E08000220704770B504460D460068066C00EB5A
:102E1800411303F530639A68A179012911D0384923
:102E28008E4256D03DB905EBC50304EB8303D3F8B6
:102E38006432002B5ED0E9B2204605F04FFE002038
:102E480070BD12F0080F09D02E498E42F7D912F43E
:102E5800004FF4D04FF400429A60F0E712F0200FD0
:102E680002D020229A60EAE712F0280FE7D125491C
:102E78008E4206D912F4004F03D04FF400429A60F4
:102E8800DDE705EBC50204EB8202D2F874121B6978
:102E9800C3F31203CB1AC2F868327DB905EBC50239
:102EA80004EB8202D2F864226AB105EBC50204EB96
:102EB8008202D2F860120B44C2F86032E9B22046AE
:102EC80005F00CFEBBE704F29C42012104F0BCFBB8
:102ED800F4E712F4004F03D04FF400429A60AEE7D3
:102EE80012F0200F01D020229A60E9B2204605F0A6
:102EF800F5FDA4E704F29C42002104F0A5FB9AE743
:102F08000A31544F0A30544F38B5044603681D6CD3
:102F180003EB4113D3F8081B0E4A954207D903F572
:102F2800306311F4004F02D04FF400429A602046FB
:102F380005F0CCFD074B9D4202D9A379012B01D0A6
:102F4800002038BD04F29C420121206804F07CFB7B
:102F5800F6E700BF0A30544F90F89434012B0CD098
:102F680010B50446012380F894344174006804F0D5
:102F7800CAFA002084F8940410BD0220704738B5BE
:102F880005468C4611F0800F29D101F00F0E0EEB8B
:102F9800CE04A40004F514740444211D0EEBCE0ED7
:102FA80000EB8E0E00208EF855020CF00F0C81F805
:102FB80000C08A600B714A780AB1A1F81AC0022BC6
:102FC8001CD095F89434012B1BD0012385F8943438
:102FD800286803F0C1FF002085F8940438BD01F08B
:102FE8000F0000EBC001890010312944043100EBC7
:102FF800C00005EB800001244475D6E700234B711F
:10300800DFE70220EAE710B504460A4611F0800F10
:1030180020D101F00F0000EBC0039B0003F51473EF
:103028002344191D00EBC00004EB8000002380F846
:10303800553202F00F020A7094F89434012B18D01C
:10304800012384F89434206803F0D4FF002084F826
:10305800940410BD01F00F0000EBC0039B00103377
:103068002344191D00EBC00004EB800001234375C5
:10307800DFE70220EDE710B5144601F00F0C0CEB6A
:10308800CC01890001F51471014404310CEBCC0E1C
:1030980000EB8E0ECEF86022CEF864320023CEF814
:1030A80068328EF855328EF854C28279012A04D0DB
:1030B800006804F085F8002010BDCEF87042F7E7EC
:1030C80001F00F0101EBC10100EB8101D1F86802A9
:1030D800704710B5144601F00F0C0CEBCC018900B9
:1030E8001031014404310CEBCC0E00EB8E0ECEF8FF
:1030F8002020CEF824300023CEF8283001238EF883
:1031080015308EF814C082799A4204D0006804F011
:1031180057F8002010BDCEF83040F7E738B501F079
:103128000F050279AA4238D304460B4611F0800FE6
:103138001FD101EBC101890001F51471014404316B
:1031480003EBC30300EB8303002283F8552201231A
:103158008B700D7094F89434012B20D0012384F8DF
:103168009434206804F074F985B1002084F894043C
:1031780038BD05EBC501890010310144043105EB68
:10318800C50300EB830301225A75E0E704F29C4271
:10319800A179206804F058FAE7E70120E8E702205F
:1031A800E6E701F00F0302799A4230D310B50446DE
:1031B80011F0800F1ED103EBC301890001F51471D2
:1031C8000144043103EBC30200EB8202002082F8C1
:1031D800550200228A700B7094F89434012B18D091
:1031E800012384F89434206804F05FF9002084F8FF
:1031F800940410BD03EBC30189001031014404316C
:1032080003EBC30200EB820201205075E1E70120C5
:1032180070470220EDE708B511F0800F0CD101F0DE
:103228000F0101EBC101890001F51471014404315A
:10323800006803F04FFF08BD01F00F0101EBC10169
:103248008900103101440431F2E72DE9F04F83B0D1
:1032580004460568284604F0B2F910B103B0BDE889
:10326800F08F0646206804F07AF90028F6D005F5B4
:103278000067BB68C3F30D23C4F8D434206804F096
:103288006EF910F0020F04D02268536903F00203AC
:103298005361206804F063F910F0100F14D022680D
:1032A800936923F010039361D5F8208008F00F0983
:1032B800C8F34343022B69D0062B00F08D802268A7
:1032C800936943F010039361206804F048F910F4FF
:1032D800002F40F09380206804F041F910F4802F0B
:1032E80040F0FC80206804F03AF90028C0F27D81A3
:1032F800206804F034F910F4006F09D0BB6813F0AB
:10330800010F40F08A812268536903F40063536116
:10331800206804F024F910F0006F15D02268536972
:1033280003F00063536194F8CC34002B40F07981AA
:10333800012184F8CC1423685B6DC3F38303C4F8BC
:10334800D034204600F0BEFA206804F008F910F4E2
:10335800805F40F06A81206804F001F910F4005F92
:1033680040F0B681206804F0FAF810F0080F40F039
:10337800C781206804F0F3F810F0800F00F0DA81BC
:10338800AB6923F08003AB610126C3E147F6F07314
:1033980018EA030F93D04FEA181B4FEAC9030193A9
:1033A80009EBC90A04EB8A0AC8F30A12DAF86012B0
:1033B800284604F023F8CBF30A0BDAF860325B44B2
:1033C800CAF86032019B4B4404EB8303D3F868329C
:1033D8005B44CAF8683272E7082204F29C41284626
:1033E80004F00CF8C8F30A1809EBC90204EB8202CE
:1033F800D2F868324344C2F8683260E7206804F0C3
:10340800B2F88046B14635E005EB49130122C3F80E
:10341800082B49462046FFF7F5FC3CE005EB49132D
:103428000822C3F8082B49462046FFF76DFD35E012
:1034380009EBC90304EB830393F85732012B41D0FE
:1034480005EB49130222C3F8082B1AF0200F04D009
:1034580005EB49132022C3F8082B1AF4005F05D0A6
:1034680005EB49134FF40052C3F8082B09F1010981
:103478004FEA5808B8F1000F3FF42DAF18F0010FCC
:10348800F4D05FFA89FB5946206804F07CF882463C
:1034980010F0010FB8D11AF0080FBFD11AF0100FB1
:1034A80004D005EB49131022C3F8082B1AF0020FB9
:1034B800CBD06B6913F0800FBAD07B6843F480637C
:1034C8007B60B5E709EBC90304EB8303002283F8AB
:1034D80057225946204605F051FBB1E7206804F011
:1034E8004AF88046B14625E05946204605F002FBD9
:1034F8001AF0080F04D005EB49130822C3F808296D
:103508001AF0100F04D005EB49131022C3F808294C
:103518001AF0400F04D005EB49134022C3F80829DC
:103528001AF0020F40D11AF0800F59D109F10109A0
:103538004FEA5808B8F1000F3FF4D4AE18F0010F65
:10354800F4D05FFA89FB5946206804F025F88246D2
:1035580010F0010FCCD009F00F03012101FA03F29A
:103568007B6B23EA02037B6305EB4913C3F8081955
:10357800A3798B42B8D109EBC90304EB8303D9695A
:103588001A6A0A441A62B9F1000FADD109EBC903EE
:1035980004EB83035B6A002BA6D104F29C42012151
:1035A800206804F051F89FE74946284603F0AEFB2F
:1035B80009EBC90304EB8303DB7D012B05D005EB85
:1035C80049130222C3F80829ADE709EBC90304EB44
:1035D80083030022DA755946204605F0D5FAEEE74E
:1035E80049462046FFF703FBA0E77B6823F0010369
:1035F8007B6094F8CC34012B08D0204605F0B8FA4B
:103608002268536903F00043536171E6002184F88E
:10361800CC14204600F056F9F2E7204605F090FA5F
:1036280071E6204605F08CFA8EE67B6823F00103EC
:103638007B601021206803F069FB1AE005EB461354
:103648004FF67F31C3F80819D3F8002922F4001285
:10365800C3F80029C3F8081BD3F8002B22F4001282
:10366800C3F8002BD3F8002B42F00062C3F8002BFC
:1036780001362379B342E1D8FB6943F00113FB61BA
:10368800E37BDBB1D7F8843043F00B03C7F8843011
:103698007B6C43F00B037B64D5F8003823F4FE639E
:1036A800C5F8003804F29C42A179206803F0CCFFE9
:1036B8002268536903F4805353614CE67A6942F2F5
:1036C8002B0313437B613B6943F00B033B61E3E747
:1036D800206803F0A9FF206803F02EFCE07126683B
:1036E80000F0D4FE0146E279304603F091FA204614
:1036F80005F011FA2268536903F40053536131E667
:10370800204605F002FA2268536903F00803536162
:103718002FE601362379B3420CD906EBC60304EB36
:10372800830393F85732012BF3D1F1B22046FFF708
:1037380072FDEEE7206803F012FF10F4801F25D118
:10374800206803F00CFF10F4001F59D0012326E075
:1037580001362379B3421BD905EB4613D3F8002968
:1037680006EBC60304EB83031B7E012BF0D1002A72
:10377800EEDA06EBC60304EB83030122DA7566F082
:103788007F01C9B22046FFF746FDE1E70126E0E7E1
:103798002268536903F480135361D1E70133227916
:1037A8009A4228D905EB4312D2F8001B03EBC30257
:1037B80004EB820292F85822012AEFD10029EDDAAF
:1037C80001F48031D4F8D42402F001029142E5D109
:1037D80003EBC30204EB8202012182F85712AA69A3
:1037E80042F08002AA616A6912F0800FD6D17B6824
:1037F80043F400737B602268536903F40013536138
:10380800206803F0ACFE10F0804F10D1206803F060
:10381800A6FE10F0040F3FF421AD23685D6815F093
:10382800040F0DD1226853682B43536016E52046D8
:1038380005F0B0F92268536903F080435361E5E766
:10384800204605F0ADF9EDE710B40468606A29B9BF
:1038580040EA0240A062002010BC70478C46A36A70
:1038680000EB1340002308E003F1400104EB810161
:10387800496800EB11400133DBB20CF1FF318B4298
:10388800F2D340EA02400CF13F0104EB81014860A9
:10389800E1E70368596200207047000003460268A8
:1038A8000121C0F8D814002083F8CC04936943F0B0
:1038B80000639361516D024B0B435365704700BF22
:1038C8000300001070470000134BDB6813F0040F6F
:1038D80007D1114BDB6803F0070383421AD001209C
:1038E800704710B50C4AD36823F007031843D0601B
:1038F800FDF7F4FD0446084B5B6813F4005F07D13D
:10390800FDF7ECFD001BB0F57A7FF4D9012000E04B
:10391800002010BD0020704700480258024AD368B2
:1039280043F08073D360704700480258002800F0C5
:10393800398338B50446036813F0010F25D0944A3B
:10394800136903F03803926A102B15D0182B0FD087
:103958006368B3F5803F3FD0002B53D18C4B1A6876
:1039680022F480321A601A6822F480221A6038E041
:1039780002F00302022AEBD1854B1B6813F4003FC7
:1039880003D06368002B00F00F83236813F0020F45
:1039980000F0A1807E4A1369926A13F038035AD066
:1039A800182B55D0E368002B00F0DE8078490A68B0
:1039B80022F0190213430B60FDF790FD0546744B86
:1039C8001B6813F0040F40F0AD80FDF787FD401B26
:1039D8000228F4D90320EEE26D4A136843F48033D9
:1039E800136063682BB3FDF779FD0546684B1B68C8
:1039F80013F4003FC9D1FDF771FD401B6428F5D9C8
:103A08000320D8E2B3F5A02F09D0614B1A6822F43D
:103A180080321A601A6822F480221A60E1E75C4B4F
:103A28001A6842F480221A601A6842F480321A60D6
:103A3800D7E7FDF753FD0546554B1B6813F4003FC8
:103A4800A3D0FDF74BFD401B6428F5D90320B2E253
:103A580012F0030FA6D14E4B1B6813F0040F03D0CE
:103A6800E368002B00F0A282494A136823F0190387
:103A7800E1680B431360FDF731FD0546444B1B68B5
:103A880013F0040F06D1FDF729FD401B0228F5D9D4
:103A9800032090E2FDF73CFD41F20303984212D85F
:103AA8002269402A07D03A494B6823F47C3343EA19
:103AB80002334B600FE0364A536823F47C3343F4F7
:103AC8000033536007E0324A536823F0FE4321690C
:103AD80043EA01635360236813F0100F00F08880F5
:103AE8002B4A136903F03803926A082B56D0182B17
:103AF80050D0E369002B00F0B880254A136843F0E2
:103B080080031360FDF7EAFC0546214B1B6813F49C
:103B1800807F40F08880FDF7E1FC401B0228F4D943
:103B2800032048E2FDF7F4FC41F20303984212D85F
:103B38002269402A07D016494B6823F47C3343EAAC
:103B480002334B60C7E7124A536823F47C3343F4CB
:103B580000335360BFE70E4A536823F0FE432169E0
:103B680043EA01635360B6E7094A136823F0010387
:103B78001360FDF7B3FC0546054B1B6813F0040FF3
:103B8800A9D0FDF7ABFC401B0228F5D9032012E2AF
:103B98000044025802F00302012AAAD1A14B1B6873
:103BA80013F4807F03D0E369802B40F00182FDF796
:103BB800AFFC41F20303984212D8226A202A07D0A8
:103BC80098494B6823F0F84343EA82634B600FE05F
:103BD800944A536823F0F84343F08043536007E066
:103BE800904AD36823F07C53216A43EA0163D36087
:103BF800236813F0080F60D06369002B49D0894A05
:103C0800536F43F001035367FDF768FC0546854B86
:103C18005B6F13F0020F50D1FDF760FC401B0228C8
:103C2800F5D90320C7E1FDF773FC41F2030398427D
:103C380012D8226A202A07D07A494B6823F0F84321
:103C480043EA82634B60D3E7764A536823F0F8432C
:103C580043F080435360CBE7724AD36823F07C5328
:103C6800216A43EA0163D360C2E76E4A136823F00E
:103C780080031360FDF732FC05466A4B1B6813F49A
:103C8800807FB5D0FDF72AFC401B0228F5D9032018
:103C980091E1644A536F23F001035367FDF71EFC5B
:103CA8000546604B5B6F13F0020F06D0FDF716FC5C
:103CB800401B0228F5D903207DE1236813F0200F6B
:103CC80029D0A3699BB1574A136843F48053136002
:103CD800FDF704FC0546534B1B6813F4005F1AD12B
:103CE800FDF7FCFB401B0228F5D9032063E14D4A90
:103CF800136823F480531360FDF7F0FB0546494B26
:103D08001B6813F4005F06D0FDF7E8FB401B022890
:103D1800F5D903204FE1236813F0040F21D1636A1A
:103D2800002B00F047813F4A126902F03802182A36
:103D380000F0EE80022B79D03A4A136823F08073A2
:103D48001360FDF7CBFB0446364B1B6813F0007F6E
:103D580000F0DC80FDF7C2FB001B0228F4D9032029
:103D680029E1314A136843F480731360FDF7B6FB09
:103D780005462D4B1B6813F4807F06D1FDF7AEFB7B
:103D8800401B6428F5D9032015E1A368012B0AD04C
:103D98000BBB244B1A6F22F001021A671A6F22F02C
:103DA80004021A6704E01F4A136F43F00103136704
:103DB800A36833B3FDF792FB05461A4B1B6F13F04C
:103DC800020FACD1FDF78AFB401B41F288339842C1
:103DD800F3D90320EFE0052B09D0124B1A6F22F01C
:103DE80001021A671A6F22F004021A67E0E70D4B06
:103DF8001A6F42F004021A671A6F42F001021A673A
:103E0800D6E7FDF76BFB0546064B1B6F13F0020F59
:103E180085D0FDF763FB401B41F288339842F3D904
:103E28000320C8E00044025800480258694A136851
:103E380023F080731360FDF751FB0546654B1B6843
:103E480013F0007F06D0FDF749FB401B0228F5D987
:103E58000320B0E05F4B996A5F4A0A40A16AE06AB2
:103E680041EA00110A439A62226B013AC2F308023E
:103E7800616B0139490289B20A43A16B013909040E
:103E880001F4FE010A43E16B0139090601F0FE4124
:103E98000A431A63DA6A22F00102DA62596B4F4A5E
:103EA8000A40A16C42EAC1025A63DA6A22F00C02A3
:103EB800216C0A43DA62DA6A22F00202616C0A4370
:103EC800DA62DA6A42F48032DA62DA6A42F400329A
:103ED800DA62DA6A42F48022DA62DA6A42F00102CD
:103EE800DA621A6842F080721A60FDF7F7FA04463F
:103EF800384B1B6813F0007F06D1FDF7EFFA001B63
:103F08000228F5D9032056E0002054E0002052E0B2
:103F1800304A916A106B012B4ED001F00303A26A5C
:103F280093424BD1C1F30511E36A994248D1C0F3DA
:103F38000802236B013B9A4244D1C0F34622636BCB
:103F4800013B9A4240D1C0F30642A36B013B9A421F
:103F58003CD1C0F30660E36B013B984238D11D4B5E
:103F68005B6BC3F3CC03A26C9A4201D1002022E020
:103F7800184AD36A23F00103D362FDF7AFFA054666
:103F8800FDF7ACFAA842FBD0124A516B134B0B4019
:103F9800A16C43EAC1035363D36A43F00103D362BC
:103FA800002008E001207047012004E0012002E021
:103FB800012000E0002038BD0120FCE70120FAE7DD
:103FC8000120F8E70120F6E70120F4E70120F2E7F5
:103FD8000120F0E7004402580CFCFFFF0700FFFF38
:103FE800F8B57E4B1B6903F03803102B00F0F28004
:103FF800182B10D013B17A4C2046F8BD774B1B68AC
:1040080013F0200F00F0E880744B1868C0F3C1006B
:10401800744CC440F0E7714B9D6A05F003059C6A37
:10402800C4F30514D86A00F001005B6BC3F3CC033A
:1040380003FB00F0FCF702FA0646002CDCD0012D49
:1040480076D0022D00F0A4800DB32046FCF7F6F9D7
:1040580001466548FCF7FEFA0446604B186BC0F34E
:104068000800FCF7EBF905464FF064513046FCF7C1
:104078003DFA01462846FCF731F94FF07E51FCF72E
:104088002DF901462046FCF731FA044671E0534BFE
:104098001B6813F0200F29D0504F3B68C3F3C103AE
:1040A8005048D840FCF7CAF905462046FCF7C6F93F
:1040B80001462846FCF7CEFA0446386BC0F30800E0
:1040C800FCF7BCF905464FF064513046FCF70EFA90
:1040D80001462846FCF702F94FF07E51FCF7FEF83E
:1040E80001462046FCF702FA044642E02046FCF767
:1040F800A5F901463D48FCF7ADFA0446374B186B65
:10410800C0F30800FCF79AF905464FF064513046B1
:10411800FCF7ECF901462846FCF7E0F84FF07E5131
:10412800FCF7DCF801462046FCF7E0F9044620E0FD
:104138002046FCF783F901462B48FCF78BFA044626
:10414800264B186BC0F30800FCF778F905464FF0CA
:1041580064513046FCF7CAF901462846FCF7BEF818
:104168004FF07E51FCF7BAF801462046FCF7BEF93D
:1041780004461A4B1B6BC3F34623581CFCF75EF925
:1041880001462046FCF766FAFCF700FB044633E7D5
:104198002046FCF753F901461548FCF75BFA04463C
:1041A8000E4B186BC0F30800FCF748F905464FF0B2
:1041B80064513046FCF79AF901462846FCF78EF818
:1041C8004FF07E51FCF78AF801462046FCF78EF93D
:1041D8000446CEE7074C0FE7024C0DE700440258AF
:1041E80000093D000090D0030024744A0024744C58
:1041F8000024F44A00127A00002800F0328170B5D9
:104208000D4604469B4B1B6803F00F038B420BD2F1
:10421800984A136823F00F030B431360136803F0E5
:104228000F038B4240F01F81236813F0040F0CD05A
:104238002269914B9B6903F070039A4205D98E4914
:104248008B6923F070031A438A61236813F0080FFF
:104258000CD06269884BDB6903F070039A4205D978
:104268008549CB6923F070031A43CA61236813F0A8
:10427800100F0CD0A269804BDB6903F4E0639A420B
:1042880005D97D49CB6923F4E0631A43CA612368E1
:1042980013F0200F0CD0E269774B1B6A03F0700310
:1042A8009A4205D974490B6A23F070031A430A62CB
:1042B800236813F0020F0CD0E2686F4B9B6903F080
:1042C8000F039A4205D96C498B6923F00F031A43EF
:1042D8008A61236813F0010F41D0674A936923F478
:1042E8007063A1680B4393616368022B0AD0032BA8
:1042F80027D0012B2CD0604A126812F0040F06D187
:104308000120ADE0126812F4003F00F0AE805A4977
:104318000A6922F0070213430B61FDF7DFF806462E
:10432800554B1B6903F038036268B3EBC20F16D014
:10433800FDF7D4F8801B41F288339842F0D9032066
:104348008EE04D4A126812F0007FE0D1012087E02C
:10435800494A126812F4807FD9D1012080E023688D
:1043680013F0020F0CD0E268434B9B6903F00F0374
:104378009A4205D240498B6923F00F031A438A6198
:104388003C4B1B6803F00F03AB420AD9394A136848
:1043980023F00F032B431360136803F00F03AB42A2
:1043A80065D1236813F0040F0CD02269324B9B6946
:1043B80003F070039A4205D22F498B6923F07003EA
:1043C8001A438A61236813F0080F0CD062692A4BDC
:1043D800DB6903F070039A4205D22749CB6923F0C1
:1043E80070031A43CA61236813F0100F0CD0A26936
:1043F800214BDB6903F4E0639A4205D21E49CB697D
:1044080023F4E0631A43CA61236813F0200F0CD029
:10441800E269194B1B6A03F070039A4205D21649E8
:104428000B6A23F070031A430A62FFF7D9FD124999
:104438008B69C3F30323114AD35C03F01F03D840ED
:104448008B6903F00F03D35C03F01F0320FA03F317
:104458000B4A13600B4B18600B4B1868FCF7DCFF1A
:1044680070BD012070470120FAE70120F8E701201C
:10447800F6E700BF0020005200440258809E000862
:1044880004000024000000240C00002408B5FFF7F5
:10449800A7FD0B4A9369C3F303230A49CB5C03F0D6
:1044A8001F0320FA03F3926902F00F02885C00F000
:1044B8001F0023FA00F0044A1060044A136008BD84
:1044C80000440258809E00080400002400000024D4
:1044D80008B5FFF7DBFF054BDB69C3F30213044A9A
:1044E800D35C03F01F03D84008BD00BF0044025846
:1044F800809E000808B5FFF7C9FF054BDB69C3F3C9
:104508000223044AD35C03F01F03D84008BD00BF50
:1045180000440258809E0008404B9B6A03F0030346
:10452800032B79D070B505460E463C4A136823F034
:1045380080631360FCF7D2FF0446384B1B6813F006
:10454800006F06D0FCF7CAFF031B022BF5D9032026
:1045580070BD324B9A6A22F47C32296842EA0132F1
:104568009A626A68013AC2F30802A96801394902E5
:1045780089B20A43E9680139090401F4FE010A43D2
:1045880029690139090601F0FE410A439A63DA6A8A
:1045980022F0C00269690A43DA62DA6A22F020026C
:1045A800A9690A43DA62DA6A22F01002DA62D96B80
:1045B8001B4A0A40E96942EAC102DA63DA6A42F050
:1045C8001002DA62C6B91A46DB6A43F40023D362E2
:1045D800124A136843F080631360FCF77FFF0446B8
:1045E8000E4B1B6813F0006F14D1FCF777FF001B0C
:1045F8000228F5D90320ABE7012E05D0074AD36A74
:1046080043F40013D362E3E7044AD36A43F4801304
:10461800D362DDE700209BE7012070470044025881
:104628000700FFFF404B9B6A03F00303032B79D07D
:1046380070B505460E463C4A136823F08053136054
:10464800FCF74CFF0446384B1B6813F0005F06D09C
:10465800FCF744FF031B022BF5D9032070BD324B36
:104668009A6A22F07C72296842EA01529A626A6860
:10467800013AC2F30802A9680139490289B20A431A
:10468800E9680139090401F4FE010A43296901397D
:10469800090601F0FE410A431A64DA6A22F440620C
:1046A80069690A43DA62DA6A22F40072A9690A437C
:1046B800DA62DA6A22F48072DA62596C1B4A0A40BA
:1046C800E96942EAC1025A64DA6A42F48072DA623B
:1046D800C6B91A46DB6A43F48003D362124A1368E8
:1046E80043F080531360FCF7F9FE04460E4B1B6839
:1046F80013F0005F14D1FCF7F1FE001B0228F5D976
:104708000320ABE7012E05D0074AD36A43F0807334
:10471800D362E3E7044AD36A43F40003D362DDE7D4
:1047280000209BE701207047004402580700FFFF64
:10473800F8B50446036813F0006F30D0836EB3F504
:10474800001F26D00ED8EBB1B3F5801F07D1022188
:104758000830FFF7E1FE054645B12E4621E0012667
:1047680035461EE0B3F5401F09D10025984A136D60
:1047780023F44013A16E0B431365002611E00126B4
:1047880035460EE0924AD36A43F40033D3620025DB
:10479800ECE702212830FFF745FF0546DCE7002655
:1047A8003546236813F4807F14D0A36D042B32D8C8
:1047B800DFE803F003232A080800854AD36A43F494
:1047C8000033D36255BB824A136D23F00703A16DF2
:1047D8000B431365236813F4007F31D0E36D802BFE
:1047E8004CD020D8002B43D0402B19D1002104F104
:1047F8000800FFF791FE05461AE0002104F10800C1
:10480800FFF78AFE0546DDE7002104F12800FFF7DF
:1048180009FF0546D6E701263546DBE72E46D9E7E8
:10482800012635460CE0C02B02D0B3F5807F1CD1A1
:104838005DBB674A136D23F4E073E16D0B431365A9
:10484800236813F4806F46D0D4F8A830B3F5800FEE
:1048580039D01FD88BB3B3F5001F18D1002104F14C
:104868000800FFF759FE05461AE001263546E7E736
:10487800574AD36A43F40033D362D9E7002104F1DD
:104888002800FFF7CFFE0546D2E72E46D8E70126D7
:10489800354620E0B3F5C00F02D0B3F5000F09D1BB
:1048A800C5B94B4A936D23F46003D4F8A8100B43A1
:1048B800936510E0012635460DE0454AD36A43F476
:1048C8000033D362ECE7002104F12800FFF7AAFEC9
:1048D8000546E5E72E46236813F4006F24D0D4F884
:1048E800AC30B3F1007F42D00ED8002B39D0B3F1F1
:1048F800807F06D1002104F10800FFF70DFE054670
:1049080008E0012635460FE0B3F1407F02D0B3F14D
:10491800806F23D1002D31D12D4A936D23F0E063B0
:10492800D4F8AC100B439365236813F0007F2ED0A6
:10493800E36C202B40D026D833B1102B20D1244A49
:10494800D36A43F40033D362002D3CD1204AD36CA0
:1049580023F03003E16C0B43D36418E0012635469D
:10496800E2E71B4AD36A43F40033D362D2E700215B
:1049780004F12800FFF756FE0546CBE72E46D3E79D
:104988000126354603E0302BDED001263546236864
:1049980013F4805F2DD0236EB3F5005F4FD019D884
:1049A800002B46D0B3F5805F0FD1002104F1080039
:1049B800FFF7B2FD054613E0022104F10800FFF7F6
:1049C800ABFD0546C0E72E46E1E70126354610E077
:1049D80000440258B3F5405F02D0B3F5804F25D1AB
:1049E800002D33D1774A136D23F4E043216E0B4336
:1049F8001365236813F4005F38D0636EB3F5003F86
:104A080053D028D843B1B3F5803F21D1012104F117
:104A18000800FFF781FD0546002D4DD1694A136D49
:104A280023F4E023616E0B4313651FE0012635462E
:104A3800DFE7644AD36A43F40033D362D0E7002146
:104A480004F12800FFF7EEFD0546C9E72E46D0E73A
:104A5800012635460AE0B3F5802FDDD0B3F5A02F47
:104A6800DAD0B3F5403FD7D001263546236813F492
:104A7800804F31D0D4F8B030B3F1005F45D020D8A2
:104A880043B1B3F1805F19D1012104F10800FFF7A8
:104A980043FD0546002D3FD14A4A936D23F0E0437C
:104AA800D4F8B0100B43936516E0012104F12800F7
:104AB800FFF7B8FD0546AFE72E46D7E7012635468E
:104AC8000AE0B3F1804FE5D0B3F1A04FE2D0B3F1E3
:104AD800405FDFD001263546236813F4004F09D024
:104AE800236FB3F1805F19D0B3F1005F24D0D3B145
:104AF80001263546236813F0807F33D0A36C032B3F
:104B08005BD8DFE803F027225327012104F12800AE
:104B1800FFF788FD0546BDE72E46DDE7294AD36A3B
:104B280043F40033D36275B9264A136D23F040531A
:104B3800216F0B431365DDE7012104F10800FFF73E
:104B4800EBFC0546EFE72E46D4E71E4AD36A43F44A
:104B58000033D362A5BB1B4AD36C23F00303A16CBB
:104B68000B43D364236813F4800F2DD1236813F00B
:104B7800010F00F0A580E36F282B00F29F80DFE88B
:104B880003F08D9D9D9D9D9D9D9D879D9D9D9D9DBA
:104B98009D9D969D9D9D9D9D9D9D8D9D9D9D9D9D54
:104BA8009D9D8D9D9D9D9D9D9D9D8D00022104F146
:104BB8000800FFF7B1FC0546CCE701263546D1E7EA
:104BC8002E46CFE700440258914A136843F4807395
:104BD8001360FCF783FC07468D4B1B6813F4807F3A
:104BE80005D1FCF77BFCC01B6428F5D90325002DF3
:104BF8004AD1884B1B6FD4F8B420534013F4407F3C
:104C08000CD0844B1A6F22F44072196F41F4803132
:104C18001967196F21F4803119671A67D4F8B4300D
:104C2800B3F5807F15D08DBBD4F8B43003F440724F
:104C3800B2F5407F1ED0774A136923F47C53136181
:104C480074490B6FD4F8B420C2F30B0213430B67FB
:104C58008CE7FCF743FC07466E4B1B6F13F0020F03
:104C6800E1D1FCF73BFCC01B41F288339842F3D9F1
:104C78000325D8E76748026922F47C52664901EAAD
:104C8800131313430361DBE72E466FE72E466DE7E8
:104C9800012104F10800FFF73FFC0546E5B95D4A2C
:104CA800536D23F03803E16F0B43536508E001218E
:104CB80004F12800FFF7B6FC0546EFE70126354664
:104CC800236813F0020F17D0A36F052B28D8DFE84D
:104CD80003F00B05200B0B0B2E46F1E7012104F125
:104CE8000800FFF719FC0546EDB94A4A536D23F051
:104CF8000703A16F0B435365236813F0040F23D0F8
:104D0800D4F89430052B45D8DFE803F0150F3D158E
:104D18001515012104F12800FFF784FC0546E3E797
:104D280001263546E8E72E46E6E7012104F10800AA
:104D3800FFF7F2FB054685BB364A936D23F0070360
:104D4800D4F894100B439365236813F0200F34D0E4
:104D5800D4F89030B3F1005F4ED023D843B1B3F10B
:104D6800805F1CD1002104F10800FFF7D5FB054640
:104D7800002D48D1274A536D23F0E043D4F8901012
:104D88000B43536519E0012104F12800FFF74AFCA1
:104D98000546D0E701263546D6E72E46D4E7012654
:104DA80035460AE0B3F1804FE2D0B3F1A04FDFD02F
:104DB800B3F1405FDCD001263546236813F0400F7D
:104DC80037D0D4F89C30B3F5006F53D026D843B110
:104DD800B3F5806F19D1002104F10800FFF79CFB9F
:104DE8000546002D4DD10B4A936D23F4E053D4F8BA
:104DF8009C100B4393651CE0022104F12800FFF787
:104E080011FC0546B4E72E46D7E70126354610E0E3
:104E18000048025800440258CFFFFF00B3F5805FF6
:104E2800DFD0B3F5A05FDCD0B3F5406FD9D0012651
:104E38003546236813F0800F33D0D4F8A030B3F58B
:104E4800804F00F0A38021D843B1B3F5005F1AD199
:104E5800002104F10800FFF75FFB0546002D40F034
:104E68009C80814A936D23F46043D4F8A0100B43CF
:104E7800936516E0022104F12800FFF7D3FB0546ED
:104E8800AFE72E46D5E7012635460AE0B3F5004FD1
:104E9800E4D0B3F5204FE1D0B3F5C04FDED0012602
:104EA8003546236813F0080F0CD0D4F88430B3F5D6
:104EB800805F74D06C4A536D23F44053D4F8841047
:104EC8000B435365236813F0100F0CD0D4F89830B7
:104ED800B3F5807F6CD0644A936D23F44073D4F8A3
:104EE80098100B439365236813F4002F0BD0D4F864
:104EF800A430B3F5803F74D0B3F5003F67D0002BE2
:104F08005FD001263546236813F4802F0CD0D4F8DF
:104F18008830B3F5001F7CD0B3F5401F6FD0B3F5D0
:104F2800801F67D001263546236813F4803F08D0D8
:104F3800236D002B76D0B3F5803F00F081800126E9
:104F48003546236813F0005F40F08380236813F42C
:104F5800003F00F08E80D4F88030B3F5807F00F0F9
:104F6800EC8040F28380B3F5007F03D0B3F5407F37
:104F780040F0E180002D40F0E6803B4A536D23F479
:104F88004073D4F880100B43536572E0022104F19A
:104F98002800FFF747FB054660E72E4681E7022118
:104FA80004F12800FFF73EFB002883D0012681E7A3
:104FB800022104F12800FFF735FB00288BD00126D9
:104FC80089E7002104F10800FFF7A6FA05467DB934
:104FD800254A936D23F44033D4F8A4100B4393650A
:104FE80091E7022104F12800FFF71CFB0546EEE7D4
:104FF8002E4688E71C4AD36A43F40033D3627DB94E
:10500800194A536D23F44013D4F888100B435365A1
:105018008AE7012104F12800FFF704FB0546EEE7C3
:105028002E4681E7104AD36A43F40033D36275B938
:105038000D4AD36C23F48033216D0B43D36480E78E
:10504800022104F10800FFF767FA0546EFE72E464C
:1050580077E7022104F12800FFF7E4FA00283FF47B
:1050680075AF012672E700BF00440258002B81D0BB
:105078000126236813F4801F06D04F4A136D23F0CE
:105088000043616F0B431365236813F0805F07D0FB
:10509800494A136923F48043D4F8B8100B431361C9
:1050A800236813F4001F06D0434A136D23F080735E
:1050B800E16E0B431365236813F0804F09D03E4B14
:1050C8001A6922F400421A611A69D4F8BC100A431A
:1050D8001A612368002B06DA374AD36C23F0405351
:1050E800616D0B43D364236813F4000F07D0324A71
:1050F800536D23F44003D4F88C100B435365636855
:1051080013F0010F21D1636813F0020F26D16368F1
:1051180013F0040F2BD1636813F0080F30D16368C4
:1051280013F0100F35D1636813F0200F3AD106B190
:1051380001263046F8BD01269BE71F4AD36A43F48F
:105148000033D36216E72E4693E7002104F10800E6
:10515800FFF7E2F90028D6D00646D4E7012104F18A
:105168000800FFF7D9F90028D1D00646CFE7022179
:1051780004F10800FFF7D0F90028CCD00646CAE7AA
:10518800002104F12800FFF74DFA0028C7D0064691
:10519800C5E7012104F12800FFF744FA0028C2D02E
:1051A8000646C0E7022104F12800FFF73BFA002871
:1051B800BDD00646BBE700BF0044025808B5FFF75C
:1051C80065F9054B1B6AC3F30213044AD35C03F069
:1051D8001F03D84008BD00BF00440258809E000845
:1051E8002DE9F0410446864B9D6A9E6AC6F3053652
:1051F800D86AC0F30010DB6BC3F3CC0303FB00F0E9
:10520800FBF71CF9002E00F0F58005F003050746B2
:10521800012D79D0022D00F0CB800DB33046FBF77D
:105228000DF901467748FBF715FA0546744B986B5C
:10523800C0F30800FBF702F906464FF06451384600
:10524800FBF754F901463046FBF748F84FF07E511A
:10525800FBF744F801462846FBF748F9054674E091
:10526800674B1B6813F0200F2CD0DFF89481D8F817
:105278000030C3F3C1036448D840FBF7DFF80546A4
:105288003046FBF7DBF801462846FBF7E3F905460D
:10529800D8F83800C0F30800FBF7D0F806464FF0FE
:1052A80064513846FBF722F901463046FBF716F8F9
:1052B8004FF07E51FBF712F801462846FBF716F926
:1052C800054642E03046FBF7B9F801464F48FBF780
:1052D800C1F905464A4B986BC0F30800FBF7AEF8D6
:1052E80006464FF064513846FBF700F90146304650
:1052F800FAF7F4FF4FF07E51FAF7F0FF014628461F
:10530800FBF7F4F8054620E03046FBF797F801462E
:105318003C48FBF79FF90546394B986BC0F30800EA
:10532800FBF78CF806464FF064513846FBF7DEF879
:1053380001463046FAF7D2FF4FF07E51FAF7CEFF1A
:1053480001462846FBF7D2F805462D4EB06BC0F350
:105358004620FBF773F84FF07E51FAF7BFFF01467E
:105368002846FBF777F9FBF711FA2060B06BC0F31A
:105378000640FBF763F84FF07E51FAF7AFFF01469E
:105388002846FBF767F9FBF701FA6060B06BC0F3DA
:105398000660FBF753F84FF07E51FAF79FFF01467E
:1053A8002846FBF757F9FBF7F1F9A060BDE8F08153
:1053B8003046FBF743F801461548FBF74BF905461D
:1053C8000F4B986BC0F30800FBF738F806464FF010
:1053D80064513846FBF78AF801463046FAF77EFFF3
:1053E8004FF07E51FAF77AFF01462846FBF77EF820
:1053F8000546AAE7002323606360A360D6E700BFE1
:10540800004402580024744A0090D0030024744CCD
:105418000024F44A2DE9F0410446864B9D6A9E6AB1
:10542800C6F30556D86AC0F300205B6CC3F3CC03FF
:1054380003FB00F0FBF702F8002E00F0F58005F002
:1054480003050746012D79D0022D00F0CB800DB35E
:105458003046FAF7F3FF01467748FBF7FBF80546B5
:10546800744B186CC0F30800FAF7E8FF06464FF0D3
:1054780064513846FBF73AF801463046FAF72EFFF2
:105488004FF07E51FAF72AFF01462846FBF72EF81F
:10549800054674E0674B1B6813F0200F2CD0DFF82B
:1054A8009481D8F80030C3F3C1036448D840FAF7B0
:1054B800C5FF05463046FAF7C1FF01462846FBF707
:1054C800C9F80546D8F84000C0F30800FAF7B6FF57
:1054D80006464FF064513846FBF708F80146304657
:1054E800FAF7FCFE4FF07E51FAF7F8FE014628461F
:1054F800FAF7FCFF054642E03046FAF79FFF0146FF
:105508004F48FBF7A7F805464A4B186CC0F308004C
:10551800FAF794FF06464FF064513846FAF7E6FF6B
:1055280001463046FAF7DAFE4FF07E51FAF7D6FE1A
:1055380001462846FAF7DAFF054620E03046FAF732
:105548007DFF01463C48FBF785F80546394B186C4A
:10555800C0F30800FAF772FF06464FF06451384668
:10556800FAF7C4FF01463046FAF7B8FE4FF07E510D
:10557800FAF7B4FE01462846FAF7B8FF05462D4E5D
:10558800306CC0F34620FAF759FF4FF07E51FAF716
:10559800A5FE01462846FBF75DF8FBF7F7F8206003
:1055A800306CC0F30640FAF749FF4FF07E51FAF726
:1055B80095FE01462846FBF74DF8FBF7E7F86060D3
:1055C800306CC0F30660FAF739FF4FF07E51FAF7F6
:1055D80085FE01462846FBF73DF8FBF7D7F8A060A3
:1055E800BDE8F0813046FAF729FF01461548FBF778
:1055F80031F805460F4B186CC0F30800FAF71EFF88
:1056080006464FF064513846FAF770FF01463046B7
:10561800FAF764FE4FF07E51FAF760FE014628461D
:10562800FAF764FF0546AAE7002323606360A360D6
:10563800D6E700BF004402580024744A0090D00303
:105648000024744C0024F44A704770477047704730
:10565800704770B504460368DE681D6915F0020FCF
:1056680010D016F0020F0DD06FF002021A6101235C
:10567800037703689B6913F0030F64D0FFF7E6FF15
:105688000023237715F0040F12D016F0040F0FD063
:1056980023686FF004021A610223237723689B6949
:1056A80013F4407F55D02046FFF7D0FF002323771F
:1056B80015F0080F12D016F0080F0FD023686FF0FE
:1056C80008021A61042323772368DB6913F0030FA8
:1056D80046D02046FFF7BAFF0023237715F0100FB6
:1056E80012D016F0100F0FD023686FF010021A6155
:1056F800082323772368DB6913F4407F37D02046DB
:10570800FFF7A4FF0023237715F0010F02D016F04E
:10571800010F33D115F4025F02D016F0800F35D196
:1057280015F4807F02D016F0800F37D115F0400FA6
:1057380002D016F0400F39D115F0200F02D016F024
:10574800200F3BD170BDFFF780FF2046FFF77FFF9A
:1057580096E72046FFF779FF2046FFF778FFA5E791
:105768002046FFF772FF2046FFF771FFB4E7204697
:10577800FFF76BFF2046FFF76AFFC3E723686FF068
:1057880001021A612046FFF75FFFC3E723686FF441
:1057980002521A61204600F0C6F9C1E723686FF487
:1057A80080721A61204600F0BFF9BFE723686FF0E6
:1057B80040021A612046FFF74BFFBDE723686FF0F0
:1057C80020021A61204600F0ADF9BBE730B5036846
:1057D8003D4A904214BF4FF0000E4FF0010EB0F159
:1057E800804F14BF72464EF00102AAB9374CA0424E
:1057F80014BF00240124364DA8420DD064B904F129
:10580800804404F58234A04214BF0024012405F525
:105818000065A84200D01CB123F070034C682343F4
:1058280012BB2A4A904214BF00220122284CA042EF
:105838001AD0CAB902F1804202F58232904214BFEE
:105848000022012204F50064A0420DD062B9214A69
:10585800904214BF0022012204F59A34A04203D0DA
:1058680012B91D4A904204D123F4407CCB6843EA24
:105878000C0323F080034A69134303608A68C262F9
:105888000A688262154A904214BF73464EF00103BB
:1058980063B9104B984214BF0023012302F57052DC
:1058A800904203D013B90C4B984201D10B690363A2
:1058B80001234361036913F0010F03D0036923F047
:1058C8000103036130BD00BF000001400008004033
:1058D8000004004000440140004801400004014029
:1058E800002852D070B50D46044690F83D30002B84
:1058F80046D0022384F83D3022689168244B0B403F
:105908009360214651F8040BFFF760FF2068816817
:105918008369026A2E680E431E491940AB68D5F8A0
:1059280018C043EA0C2343EA010C1B4B0CEA03039F
:10593800E968D5F81CC041EA0C2119432B6A1B03FE
:10594800D5F810C043EA0C130B4322F0AA016A6889
:105958006D6942EA05120A43866021688B612368F3
:105968001A62012384F8483084F83E3084F83F30C6
:1059780084F8443084F8453084F83D30002070BD08
:1059880080F83C30FBF732FCB3E70120704700BFDA
:10599800F8BFFEFFFCFCFFFF0303FFFF01F01F0140
:1059A800012303FA01FC036A23EA0C030362036A76
:1059B80002FA01F10B430362704738B5044690F8C8
:1059C8003E30DBB290F83F205FFA82FC90F844202A
:1059D800D0B294F845200D46B1B9012808BF012B73
:1059E80047D1022384F83E3084F844307DB3042D37
:1059F80039D0012200212068FFF7D0FF01220421BD
:105A08002068FFF7CBFF27E0D2B2042914D0BCF1FD
:105A1800010F08BF012B30D1013A18BF012201281C
:105A28002DD162BB022384F83E3084F83F3084F8DD
:105A3800443084F84530D9E7012A08BFBCF1010F8A
:105A480019D1022384F83F3084F84530CEE701228B
:105A580000212068FFF7A2FF2268136843F00103C2
:105A68001360002038BD012204212068FFF796FF4B
:105A7800F2E70120F6E70120F4E70120F2E7012030
:105A8800F0E7000090F83C30012B45D070B40123BA
:105A980080F83C30022380F83D3003685A689C68DF
:105AA8001E4E1F4DAB4218BFB34203D122F4700201
:105AB8004D682A4322F070020D682A435A60036831
:105AC800164AB3F1804F18BF934217D0A2F57C4213
:105AD800934213D002F5806293420FD002F58062A0
:105AE80093420BD002F57842934207D0A2F56C425C
:105AF800934203D002F59432934204D124F08004F7
:105B08008A6814439C60012380F83D30002380F8A4
:105B18003C30184670BC70470220704700000140B6
:105B2800000401407047704770470000026852E85F
:105B3800003F23F4907342E800310029F6D102684F
:105B480002F1080353E8001F0D4B0B40083242E8EE
:105B580000310029F3D1C36E012B06D02023C0F8F1
:105B68008C300023C36643677047026852E8003FE1
:105B780023F0100342E800310029F6D1EEE700BF18
:105B8800FEFFFFEF704708B5026852E8003F23F0B8
:105B9800400342E800310029F6D12023C0F88830BC
:105BA80000238367FFF7EEFF08BD704708B5806BD9
:105BB8000023A0F85E30A0F85630FFF7F6FF08BDC6
:105BC8007047000070B504460168CB6908688D68A5
:105BD80040F60F021A4008D113F0200F05D010F03C
:105BE800200F34D115F0805F31D12AB18B4A2A4079
:105BF80033D18B4E304230D1E26E012A00F0C6809C
:105C080013F4801F03D015F4800F40F09B8113F02C
:105C1800800F07D010F0800F40F09B8115F4000F23
:105C280040F0978113F0400F03D010F0400F40F080
:105C3800978113F4000F03D010F0804F40F0948147
:105C480013F0807F02D00028C0F2928170BD636F8C
:105C5800002BFBD020469847F8E713F0010F09D036
:105C680010F4807F06D001260E62D4F890103143DC
:105C7800C4F8901013F0020F0BD015F0010F08D0E4
:105C8800216802260E62D4F8901041F00401C4F88D
:105C9800901013F0040F0BD015F0010F08D02168F5
:105CA80004260E62D4F8901041F00201C4F8901056
:105CB80013F0080F0BD010F0200F00D13AB1226872
:105CC80008211162D4F890200A43C4F8902013F4F4
:105CD800006F0CD010F0806F09D022684FF400617B
:105CE8001162D4F8902042F02002C4F89020D4F831
:105CF8009020002AAAD013F0200F09D010F0200F0E
:105D080002D115F0805F03D0636F0BB1204698472E
:105D1800D4F8902023689B6813F0400F02D112F04A
:105D2800280F2CD02046FFF701FF23689B6813F04B
:105D3800400F20D0226802F1080353E8003F23F007
:105D48004003083242E800310029F3D1D4F880300A
:105D58006BB1344A1A65D4F88000FCF751F9002871
:105D68003FF474AFD4F88000036D98476EE720467F
:105D7800FFF71BFF6AE72046FFF717FF66E7204695
:105D8800FFF713FF0023C4F890305FE713F0100FFC
:105D98003FF436AF10F0100F3FF432AF10230B6210
:105DA80023689B6813F0400F00F09280D4F880209D
:105DB80013681D481D498B4218BF834238D01831DB
:105DC8008B4235D018318B4232D018318B422FD0CC
:105DD80018318B422CD018318B4229D018318B4284
:105DE80026D001F556718B4222D018318B421FD034
:105DF80018318B421CD018318B4219D018318B4284
:105E080016D018318B4213D018318B4210D018316C
:105E18008B420DD05B689BB20CE000BF0100001004
:105E280020010004B55B0008100002402800024071
:105E38005B689BB2002B3FF409AFB4F85C10994241
:105E48007FF604AFA4F85E30D369B3F5807F32D013
:105E5800226852E8003F23F4807342E800310029A9
:105E6800F6D1226802F1080353E8003F23F001034A
:105E7800083242E800310029F3D1226802F1080310
:105E880053E8003F23F04003083242E8003100297C
:105E9800F3D12023C4F88C300023E366226852E84B
:105EA800003F23F0100342E800310029F6D1D4F86E
:105EB8008000FBF705FF02232367B4F85C10B4F8F1
:105EC8005E309BB2C91A89B22046FFF779FEBDE65B
:105ED800B4F85C10B4F85E309BB2C91A89B2B4F851
:105EE8005E309BB2002B3FF4B1AE00293FF4AEAE5A
:105EF800226852E8003F23F4907342E800300028FB
:105F0800F6D1226802F1080353E8000F1A4B034048
:105F1800083242E800300028F3D12023C4F88C303E
:105F28000023E3666367226852E8003F23F010030A
:105F380042E800300028F6D1022323672046FFF705
:105F48003FFE83E64FF480130B62204600F07CFD91
:105F58007CE6A36F002B3FF479AE2046984775E6A0
:105F68002046FFF710FE71E6204600F06FFD6DE653
:105F7800204600F06AFD69E6FEFFFFEF70B586B0C7
:105F88000446016883680269134342691343C2697E
:105F980013430868884A024013430B602268536819
:105FA80023F44053E1680B435360A1692268834B93
:105FB8009A4201D0236A19439068814B03400B43EE
:105FC80093602268D36A23F00F03616A0B43D3629C
:105FD80022687C4B9A4221D07B4B9A4200F08C80FD
:105FE8007A4B9A4200F0A280794B9A4200F0B58031
:105FF800784B9A4200F0C880774B9A4200F0F480C0
:10600800764B9A4200F01981754B9A4200F02C8128
:106018006A4B9A4200F03F81802333E0714B5B6DFD
:1060280003F03803282B65D8DFE813F02900640053
:106038006400640064006400640064004D0164004E
:106048006400640064006400640064002B00640061
:106058006400640064006400640064005E0064001E
:10606800640064006400640064006400600064000C
:10607800640064006400640064006400620001233A
:1060880000E008234D498A4200F02F81E069B0F50D
:10609800004F00F0AF81202B00F20782202B00F286
:1060A8005182DFE813F01E0224024F024F0227023A
:1060B8004F024F024F022C024F024F024F024F0273
:1060C8004F024F024F0231024F024F024F024F025E
:1060D8004F024F024F024F024F024F024F024F0230
:1060E8004F024F024F023D021023CBE72023C9E79E
:1060F8004023C7E78023C5E73A4B5B6D03F00703EE
:10610800052B11D8DFE813F00600E10008000A00AB
:106118000C000E000023B5E70823B3E71023B1E70E
:106128002023AFE74023ADE78023ABE72D4B5B6D22
:1061380003F00703052B0ED8DFE803F003C90507B2
:10614800090B00239EE708239CE710239AE72023E6
:1061580098E7402396E7802394E7224B5B6D03F092
:106168000703052B0ED8DFE803F003B40507090B76
:10617800002387E7082385E7102383E7202381E7A7
:1061880040237FE780237DE7164B5B6D03F0070311
:10619800052B0ED8DFE803F0039F0507090B002342
:1061A80070E708236EE710236CE720236AE7402393
:1061B80068E7802366E700BFF369FFCF000C00584B
:1061C800FFF4FF1100100140004400400048004067
:1061D800004C00400050004000140140007800408E
:1061E800007C0040004402587D4B5B6D03F038038F
:1061F800282B20D8DFE803F0151F1F1F1F1F1F1FA4
:10620800711F1F1F1F1F1F1F171F1F1F1F1F1F1F4C
:10621800191F1F1F1F1F1F1F1B1F1F1F1F1F1F1F90
:106228001D0001232EE708232CE710232AE720234B
:1062380028E7402326E7802324E7694B5B6D03F0BA
:106248000703052B0ED8DFE803F0034A0507090BFF
:10625800002317E7082315E7102313E7202311E786
:1062680040230FE780230DE75D4B5B6D03F00703C9
:10627800052B0ED8DFE803F003350507090B0023CB
:1062880000E70823FEE61023FCE62023FAE6402375
:10629800F8E68023F6E603F50E339B6D03F007035B
:1062A800052B0ED8DFE803F0031F0507090B0223AF
:1062B800E8E60823E6E61023E4E62023E2E64023A6
:1062C800E0E68023DEE60423DCE60423DAE60423A2
:1062D800D8E60423D6E60423D4E60423D2E604232E
:1062E800D0E60423CEE60423CCE6202B27D8022BC5
:1062F800C0F01A81023B1E2B00F21881DFE813F070
:106308005000160156001601160116015B00160111
:106318001601160116011601160116016000160174
:1063280016011601160116011601160116011601AD
:106338001601160116011601160116016C00402BF4
:106348002CD14FF40040626A264B33F81220B0FB80
:10635800F2F3656805EB4501994200F2E980B3EB79
:10636800053F00F2E780002633463146FAF72EFA59
:10637800090241EA106100026B08C0182A46334638
:1063880041F10001FAF722FAA0F54072164B9A4241
:1063980000F2D2802368D8603046D4E00120D2E0F1
:1063A800FEF70CFF0028CED10020CCE003A8FEF7B2
:1063B80017FF0498F6E76846FFF72CF80198F1E70D
:1063C800074B1B6813F0200F08D0054B1B68C3F35D
:1063D800C1030648D840E5E70548B4E70348B2E7F3
:1063E80000440258989E0008FFFC0F000090D0035C
:1063F80000093D00202B15D8202B00F29F80DFE8F4
:1064080003F031379D9D3A9D9D9D3F9D9D9D9D9D8E
:106418009D9D449D9D9D9D9D9D9D9D9D9D9D9D9DFD
:106428009D9D5000402B1BD1626A4D4B33F81230B2
:10643800B0FBF3F06268530803EB4000B0FBF2F0E6
:10644800A0F110024FF6EF739A4279D883B223F085
:106458000F03C0F3420018432368D860002072E09D
:10646800012070E0FEF734F80028DDD100206AE052
:10647800FEF740F8F8E703A8FEF7B2FE0498F3E742
:106488006846FEF7C7FF0198EEE7364B1B6813F026
:10649800200F08D0334B1B68C3F3C1033248D840E0
:1064A800E2E73248C0E73048BEE7402B17D14FF447
:1064B8000040626A2A4B33F81230B0FBF3F063688D
:1064C80000EB5300B0FBF3F0A0F110024FF6EF73AE
:1064D8009A4242D8236880B2D860002033E0012075
:1064E80031E0FDF7F5FF0028E3D100202BE0FEF7AF
:1064F80001F8F8E703A8FEF773FE0498F3E7684687
:10650800FEF788FF0198EEE7164B1B6813F0200F83
:1065180008D0144B1B68C3F3C1031348D840E2E703
:106528001248C6E71048C4E701200CE001200AE041
:10653800012008E0012006E0012004E0012002E03B
:10654800012000E001200123A4F86A30A4F8683093
:1065580000236367A36706B070BD0120F3E700BF9F
:10656800989E0008004402580090D00300093D009E
:10657800836A13F0080F06D00268536823F40043B7
:10658800816B0B435360836A13F0010F06D00268D6
:10659800536823F40033C16A0B435360836A13F0D2
:1065A800020F06D00268536823F48033016B0B4353
:1065B8005360836A13F0040F06D00268536823F40B
:1065C8008023416B0B435360836A13F0100F06D08E
:1065D8000268936823F48053C16B0B439360836A0A
:1065E80013F0200F06D00268936823F40053016C5F
:1065F8000B439360836A13F0400F0AD00268536814
:1066080023F48013416C0B435360436CB3F5801F34
:106618000BD0836A13F0800F06D00268536823F406
:106628000023C16C0B43536070470268536823F41E
:10663800C003816C0B435360EBE72DE9F843054633
:106648000E4617469946DDF820802C68E46936EA3C
:1066580004030CBF4FF0010C4FF0000CBC453AD1BD
:10666800B8F1FF3FF1D0FAF739FFA0EB0900404538
:1066780034D8B8F1000F33D02B681A6812F0040F21
:10668800E3D0B6F1400218BF0122802EDDD0002AE7
:10669800DBD0DA6912F0080F11D1DA6912F4006F51
:1066A800D3D04FF400621A622846FFF73FFA20233E
:1066B800C5F89030002385F8843003200CE00824C6
:1066C8001C622846FFF732FAC5F89040002385F887
:1066D8008430012000E00020BDE8F8830320FBE7B8
:1066E8000320F9E72DE9F04182B01E46D0F8883042
:1066F800202B5BD104460D469046002A18BF00297E
:1067080001D1012053E00023C0F890302123C0F8C4
:106718008830FAF7E3FE0746A4F85480A4F85680B8
:10672800A368B3F5805F02D04FF0000816E0236934
:1067380043B34FF0000811E02023C4F88830032049
:1067480035E038F8023B2268C3F308039362B4F8D3
:10675800562092B2013A92B2A4F85620B4F85630B4
:106768009BB293B100963B46002280212046FFF75A
:1067780064FF0028E0D1002DE3D015F8012B236831
:106788009A62E4E7A8460025E8E700963B4600221F
:1067980040212046FFF751FF18B92023C4F888305C
:1067A80005E02023C4F88830032000E0022002B06E
:1067B800BDE8F0812DE9F04383B01E46D0F88C3057
:1067C800202B7ED104460D469046002A18BF00298A
:1067D80001D1012076E00023C0F890302222C0F8D1
:1067E8008C20C366FAF77AFE0746A4F85C80A4F802
:1067F8005E80A368B3F5805F06D0A3B9226972B939
:10680800FF22A4F8602014E0226922B940F2FF12A6
:10681800A4F860200DE0FF22A4F8602009E07F22A0
:10682800A4F8602005E0B3F1805F0AD00022A4F844
:106838006020B4F86080B3F5805F0CD04FF0000999
:1068480024E022691AB97F22A4F86020F1E73F22E8
:10685800A4F86020EDE7236913B14FF0000915E0B3
:10686800A946002512E02023C4F88C30032029E033
:1068780023685A6A5FFA88F3134005F8013BB4F8B5
:106888005E2092B2013A92B2A4F85E20B4F85E306B
:106898009BB28BB100963B46002220212046FFF791
:1068A800CCFE0028DFD1002DE2D123685B6A08EA1C
:1068B800030329F8023BE2E72023C4F88C300020C8
:1068C80000E0022003B0BDE8F08330B583B0044691
:1068D8000023C0F89030FAF701FE054622681268D6
:1068E80012F0080F10D123681B6813F0040F28D189
:1068F8002023C4F88830C4F88C300020E066206774
:1069080084F8840003B030BD6FF07E4300930346E3
:1069180000224FF400112046FFF78FFE0028E2D036
:10692800226852E8003F23F0800342E80031002942
:10693800F6D12023C4F88830002384F8843003205B
:10694800E0E76FF07E4300932B4600224FF480016E
:106958002046FFF772FE0028CAD0226852E8003F9E
:1069680023F4907342E800310029F6D1226802F13D
:10697800080353E8003F23F00103083242E80031DE
:106988000029F3D12023C4F88C30002384F8843004
:106998000320B7E778B310B50446D0F888300BB3B6
:1069A8002423C4F888302268136823F00103136095
:1069B800A36AE3B92046FFF7E1FA012811D022685B
:1069C800536823F4904353602268936823F02A03A2
:1069D80093602268136843F0010313602046FFF7B1
:1069E80074FF10BD80F88430FAF774FCD8E72046AD
:1069F800FFF7BEFDDEE7012070470000436E2BB9AC
:106A08000123A0F86A30A0F86830704730B40368F2
:106A18009A68C2F342629968490F094D6B5C1B0181
:106A2800084C615C93FBF1F3A0F86A30AB5C1B0186
:106A3800A25C93FBF2F3A0F8683030BC704700BF4B
:106A4800B89E0008B09E000870477047704790F8DD
:106A58008430012B18D0012380F884302423C0F817
:106A6800883003681A68196821F00101196022F05A
:106A780000520023436601680A602022C0F888207B
:106A880080F88430184670470220704738B590F86F
:106A98008430012B1DD00446012380F88430242340
:106AA800C0F8883003681D681A6822F001021A606D
:106AB8000268936823F0604319439160FFF79EFFD3
:106AC80023681D602023C4F88830002084F88400DF
:106AD80038BD0220FCE738B590F88430012B1DD072
:106AE8000446012380F884302423C0F888300368E2
:106AF8001D681A6822F001021A600268936823F080
:106B0800606319439160FFF779FF23681D602023B4
:106B1800C4F88830002084F8840038BD0220FCE7DF
:106B280082B000230193019B01330193019BB3F1D0
:106B3800706F15D80369002BF5DA002301930369F8
:106B480043F001030361019B01330193019BB3F1FE
:106B5800706F08D8036913F0010FF4D1002000E02A
:106B6800032002B070470320FBE7000084B010B593
:106B7800044603A880E80E009DF81130012B1FD1B0
:106B8800A36B23F48033A363E2681F4B1340E360D5
:106B9800E36823F44013E3609DF81830012B0AD012
:106BA8002046FFF7BDFF9DF80E30012B1CD0BDE835
:106BB800104004B07047E36843F48013E360EFE7E4
:106BC800E36843F04003E3602046FFF7A9FF9DF820
:106BD800153023B9A36B43F48033A363E3E7A36BB6
:106BE80023F48033A363DEE7E36D9BB2E365E26DD4
:106BF800064B1343E365A36843F00603A360A36849
:106C080043F02003A360D2E7BFFFBDFF0000EE03FF
:106C1800022A0AD00921C26822F47052C260C368ED
:106C280043EA8123C36000207047204B0B44204A6D
:106C3800934229D91F4B0B441F4A934226D91F4B15
:106C48000B441F4A934223D91E4B0B441E4A9342BE
:106C580020D31E4B0B441E4A93421DD91D4B0B4497
:106C68001D4A93421AD31D4B0B441D4A934217D316
:106C78001C4B0B441C4A934214D31C4B0B441C4A18
:106C8800934211D20721C6E70F21C4E70E21C2E7BC
:106C98000D21C0E70C21BEE70B21BCE70A21BAE7AA
:106CA8000921B8E70821B6E70621B4E7405327FFD2
:106CB800FF340C00401E1BFF3F420F0000DC0BFF9F
:106CC8007F4F1200808CF9FE20D6130060B6E5FED7
:106CD8005FE3160000D3CEFE40771B00C05BB3FE17
:106CE800C091210000CA91FE20753800E05459FE79
:106CF800E09C4100836843F00103836000207047F3
:106D0800836823F0010383600020704782B000236A
:106D18000193019B01330193019BB3F1706F15D867
:106D28000369002BF5DA00230193890141F0200162
:106D38000161019B01330193019BB3F1706F08D886
:106D4800036913F0200FF4D1002000E0032002B003
:106D580070470320FBE782B000230193019B0133B6
:106D68000193019BB3F1706F13D80369002BF5DA17
:106D78000023019310230361019B01330193019BBD
:106D8800B3F1706F08D8036913F0100FF4D1002025
:106D980000E0032002B070470320FBE7D0F800387A
:106DA8001943C0F8001800207047000084B0F8B5F7
:106DB800044607A880E80E00002306E003F140021D
:106DC80004EB82020021516001330E2BF6D99DF8A5
:106DD800266006BBD4F8043843F00203C4F804382C
:106DE800A36B23F40013A363236843F040032360D9
:106DF800236843F0800323600023C4F8003E9DF815
:106E08002130012B11D19DF81F304BB900212046AC
:106E1800FFF7C4FF0DE0A36B43F40013A363EBE794
:106E280001212046FFF7BAFF03E003212046FFF7C0
:106E3800B5FF10212046FFF769FF054600B101257F
:106E48002046FFF788FF00B1012504F5006C0023F8
:106E5800CCF81030CCF81430CCF81C300AE0CBB9A0
:106E68004FF00060C2F8000900220A614FF67F3235
:106E78008A6001339DF81C10994210D904EB431223
:106E880002F51061D2F800090028E8DB0020C2F8FA
:106E98000009E9E74FF09040C2F80009E4E7002351
:106EA8000AE0BBB14FF09047C2F8007B00220261B4
:106EB8004FF67F3282600133994210D904EB4312B6
:106EC80002F53060D2F8007B002FEADB0027C2F819
:106ED800007BEBE74FF00067C2F8007BE6E7DCF8E1
:106EE800103023F48073CCF810300023A3616FF0C6
:106EF800804363619DF81E301BB9A36943F01003FA
:106F0800A361A2690A4B1343A3619DF822301BB108
:106F1800A36943F00803A361012E04D02846BDE805
:106F2800F84004B07047A269024B1343A361F5E728
:106F380000383C8004000040D0F8083813F00603FD
:106F480005D0062B18BF022B03D102207047002062
:106F580070470F207047000010B591F800C04B78BB
:106F6800012B21D000F5006ED0F81C380CF00F046E
:106F78000122A24043EA0243C0F81C3800EB4C103F
:106F8800D0F8003B13F4004F0CD1D0F8002B8B68DD
:106F9800C3F30A03097943EA81431343144A1A43A2
:106FA800C0F8002B002010BDD0F81C280CF00F0EE4
:106FB80003FA0EF39BB21343C0F81C3800EB4C10D5
:106FC800D0F8003913F4004FECD1D0F800298B68C1
:106FD800C3F30A03097943EA814343EA8C5C42EA32
:106FE8000C0C034B4CEA0303C0F80039DAE700BF86
:106FF8000080001030B40B784A78012A26D000EBC4
:107008004313D3F8002B002A52DBD0F83C480A7807
:1070180002F00F024FF0010C0CFA02F224EA0242CD
:10702800C0F83C28D0F81C28097801F00F010CFAA8
:1070380001FC22EA0C42C0F81C28D3F8001B234AA2
:107048000A40C3F8002B002030BC704700EB431304
:10705800D3F80029002A1EDBD0F83C580A7802F041
:107068000F02012404FA02F292B225EA0202C0F8E1
:107078003C28D0F81C28097801F00F018C40A4B2F4
:1070880022EA0404C0F81C48D3F80019104A0A4040
:10709800C3F80029D7E7D3F8002942F00062C3F803
:1070A8000029D3F8002942F08042C3F80029D3E729
:1070B800D3F8002B42F00062C3F8002BD3F8002B62
:1070C80042F08042C3F8002B9FE700BF0078F3EF3F
:1070D800007833EC10B483B002460023019348785B
:1070E80001280AD00B7802EB4313D3F8000B0028D1
:1070F8002CDB002003B010BC70470B7802EB431365
:10710800D3F80049002C01DB0020F3E7D3F800494D
:1071180044F00064C3F800490B7802EB4313D3F83A
:10712800004944F08044C3F80049019B01330193AE
:10713800019C42F210739C42DCD80B7802EB43139B
:10714800D3F80039002BF0DB0020D3E7D3F8000B8D
:1071580040F00060C3F8000B0B7802EB4313D3F840
:10716800000B40F08040C3F8000B019B01330193F2
:10717800019842F21073984208D80B7802EB431337
:10718800D3F8003B002BF0DB0020B3E70120B1E788
:1071980010B59DF8084084B903334FEA930E4FF0B9
:1071A800000C08E000EB023303F5805351F8044B60
:1071B8001C600CF1010CF445F4D3002010BD000054
:1071C800F0B583B00C784B78012B2DD000EB441C24
:1071D8000CF530631E69864D35401D611E69854D6D
:1071E80035401D61002C40F0C7800C690CB18C68DB
:1071F8000C618C680C621D69C4F312042C431C6179
:107208001C6944F400241C61012A00F0D8800B7921
:10721800012B00F0DA80DCF8003B43F00443CCF8A3
:10722800003B002003B0F0BD0B6973BB00EB4413B7
:10723800D3F810696F4D3540C3F81059D3F8105979
:1072480045F40025C3F81059D3F81069684D354046
:10725800C3F81059012A4DD000EB4414D4F8003972
:1072680043F00443C4F800390B79012B6BD00B6948
:10727800002BD6D0D0F834380A7802F00F0101225A
:107288008A401343C0F83438CBE700EB441303F5C6
:1072980010631E69564D35401D611E69554D3540B8
:1072A8001D61D4B90E698D68AE4200D90D611D69A2
:1072B80045F400251D611D690E69C6F312063543A4
:1072C8001D610D79012DC5D11D6925F0C0451D61D0
:1072D8001D6945F000551D61BCE71E690D698F6881
:1072E8003D44013DB5FBF7F5434F07EAC545354336
:1072F8001D61E0E7CB691BB100EB4412C2F81439F9
:107308000B79012B08D000EB4410D0F8003943F07A
:107318000443C0F8003984E7D0F8083813F4807FB4
:1073280008D100EB4412D2F8003943F00053C2F8F8
:107338000039E8E700EB4412D2F8003943F08053F3
:10734800C2F80039DFE7D0F8083813F4807F0CD191
:10735800D4F8003943F00053C4F8003900920B8A7E
:107368000A78C968FFF714FF5BE7D4F8003943F0DF
:107378008053C4F80039F1E70C6954B91C698D6869
:10738800C5F312052C431C611C6944F400241C61DC
:107398003AE78D682C44013CB4FBF5F4A4B204FB35
:1073A80005F50D621D69144E06EAC4442C431C61A0
:1073B8001C690D6AC5F312052C431C6124E7CA68D1
:1073C800002A3FF424AF5A6121E7D0F8083813F4B3
:1073D800807F06D1DCF8003B43F00053CCF8003B3B
:1073E80019E7DCF8003B43F08053CCF8003B12E788
:1073F8000000F8FFFFFF07E00000F81F00B583B0AA
:10740800844608464FEA920E02F00302002305E084
:107418000CF58051096840F8041B01337345F7D314
:107428009AB10CF5805CDCF8003001934FF0000C49
:107438005FFA8CF3D900019BCB4000F8013B0CF1BB
:10744800010C013A92B2002AF2D103B05DF804FBB4
:107458000B784A78012A14D000EB4310D0F8002B9F
:10746800002A06DB2BB1D0F8003B23F08043C0F89C
:10747800003BD0F8003B43F40013C0F8003B002069
:10748800704700EB4310D0F80029002A06DB2BB127
:10749800D0F8003923F08043C0F80039D0F800391B
:1074A80043F40013C0F80039E9E70B784A78012A59
:1074B8000ED000EB4310D0F8003B23F40013C0F8C3
:1074C800003B0B79023BDBB2012B15D9002070473A
:1074D80000EB4310D0F8003923F40013C0F800394A
:1074E8000B79023BDBB2012BF0D8D0F8003943F01E
:1074F8008053C0F80039E9E7D0F8003B43F08053E7
:10750800C0F8003BE2E7D0F8003823F4FE63C0F887
:107518000038D0F80038090101F4FE611943C0F8B9
:10752800001800207047D0F8003E23F00303C0F88D
:10753800003ED0F8043823F00203C0F804380020D5
:107548007047D0F8003E23F00303C0F8003ED0F89F
:10755800043843F00203C0F8043800207047426939
:10756800806910407047D0F8183800F50060C0698D
:107578001840000C7047D0F8183800F50060C06952
:10758800184080B2704700EB4111D1F8082B00F584
:10759800006040691040704710B4D0F81048D0F827
:1075A800343801F00F02D340DB01DBB2234300EB98
:1075B800411000F510608068184010BC70474069A1
:1075C80000F00100704738B50546C36823F0C04392
:1075D800C360012913D019BBC36843F08043C3605B
:1075E80000240A20F9F780FF0A342846FFF7E7FF4E
:1075F80008B1C72CF5D9C82C14D0002038BDC368F1
:1076080043F00053C36000240A20F9F76DFF0A34E1
:107618002846FFF7D4FF0128EDD0C72CF4D9EAE7B4
:107628000120EBE70120E9E7D0F80029054B1340DA
:10763800C0F80039D0F8043843F48073C0F804382F
:107648000020704700F8FFFF10B4046C144B9C42F4
:1076580003D9D0F8003B002B16DB0024C0F8104BF0
:10766800D0F8104B44F40024C0F8104BD0F8104B5D
:1076780044F01804C0F8104BD0F8104B44F0C04444
:10768800C0F8104B012902D0002010BC7047C0F888
:10769800142BD0F8003B43F08023C0F8003BF3E7FD
:1076A8000A30544F10B5D0F8D43203F1B00250F874
:1076B80022408CB100EB820043687BB194F8000251
:1076C800FF280DD09B6894F8012221469847FF2394
:1076D80084F80032002010BD0320FCE70020FAE700
:1076E8000020F8E70A230380004870478C00002434
:1076F800F8B506460F4F8221384600F041FC054692
:107708000121384600F03CFC04468121384600F04F
:1077180037FC0DB11022AA711CB14022227100223F
:10772800627118B1402202710022427143233380F2
:107738000048F8BD48000024F8B506460F4F8221DE
:10774800384600F01DFC05460121384600F018FCBB
:1077580004468121384600F013FC0DB11022AA71AD
:107768001CB1402222710022627118B140220271BC
:1077780000224271432333800048F8BD48000024AA
:10778800F8B506460F4F8221384600F0F9FB05464A
:107798000121384600F0F4FB04468121384600F008
:1077A800EFFB0DB11022AA711CB100222271022236
:1077B800627118B1002202710222427143233380A0
:1077C8000048F8BD4800002438B5D0F8D432B033AA
:1077D80050F8235095B1044601F036FAC5F80C026A
:1077E800D4F8D432B03304EB83046368DB6805F55E
:1077F8000371D5F804029847002038BD0320FCE740
:1078080038B5D0F8C852D0F8D432B03350F8234045
:1078180084B301F00F0303EB830200EB8202926949
:107828004AB103EBC30C05EB8C05ED69B2FBF5FC23
:1078380005FB1C2292B10023C4F81432D0F8D432CC
:10784800B03300EB830043681B69ABB10A4604F50B
:107858000471D4F808029847002038BD03EB83036D
:1078680000EB830300249C612346224601F034FA8E
:107878002046F2E70320F0E70020EEE7F0B583B0FA
:10788800D0F8D43203F1B00250F8227000228DF8FB
:107898000720ADF80420002F7BD004460D46097858
:1078A80011F0600634D0202E6CD1EA882AB311F08A
:1078B800800F07D16B7887F80032EA883F2A13D8FF
:1078C800D2B212E0B03300EB83035B689B683946A1
:1078D80068789847EA88072A28BF07223946204649
:1078E80000F005FF002651E0402287F801223946C2
:1078F800204600F011FF002648E0B03300EB830477
:1079080063689B68002229466878984700263DE00E
:107918006F780B2F31D8DFE807F006393030303078
:1079280030303030162690F89C32DBB2032B04D06E
:10793800294600F062FB032628E0022201A900F094
:10794800D6FE3E4622E090F89C32DBB2032B04D0F0
:10795800294600F052FB032618E001220DF1070129
:1079680000F0C5FE12E090F89C32DBB2032B0DD07C
:10797800294600F042FB032608E0294600F03DFBBB
:10798800032603E0294600F038FB0326304603B0FF
:10799800F0BD0326FAE738B50446812101F07CF9E9
:1079A800002525870121204601F076F9A4F87851B1
:1079B8008221204601F070F9A4F84C50A4F84E50EA
:1079C800D4F8D43203F1B00254F822209AB1B0337B
:1079D80004EB83035B685B689847D4F8D432B03310
:1079E80054F8230001F03AF9D4F8D432B03344F80B
:1079F8002350C4F8BC52002038BD70B504464FF47B
:107A0800077001F027F9002849D005464FF407729E
:107A1800002101F09BF9D4F8D432B03344F8235054
:107A2800C4F8BC52237C002B41D14FF400730222CE
:107A38008121204601F025F9012626874FF400739D
:107A480002223146204601F01CF9A4F8786110237F
:107A5800A4F84E30082303228221204601F011F9B0
:107A68000123A4F84C300026C5F80462D4F8D432B7
:107A7800B03304EB83035B681B689847C5F814624E
:107A8800C5F81862D5F8042262B3257C1DBB4FF4F3
:107A980000730121204601F027F9284670BDD4F86B
:107AA800D432B033002244F823200225F5E74023DE
:107AB80002228121204601F0E4F80126268740238E
:107AC80002223146204601F0DCF8A4F87861102340
:107AD800A4F84E30BEE740230121204601F004F906
:107AE8000025DAE70225D8E739B1D0F8D432B03327
:107AF80000EB830041600020704703207047D0F8F6
:107B0800D432B03350F823302BB1C3F80812C3F87D
:107B180010220020704703207047D0F8D432B033C9
:107B280050F823301BB1C3F804120020704703201B
:107B3800704708B5D0F8D432B03350F823209AB142
:107B4800D2F814320BB1012008BD0123C2F8143257
:107B5800D2F81032C362D2F81032D2F8082281214A
:107B680001F0BAF80020EFE70320EDE710B5D0F8F0
:107B7800D432B03350F8232092B1047C44B94FF486
:107B88000073D2F80422012101F0AEF8204610BD9E
:107B98004023D2F80422012101F0A6F80024F5E7D9
:107BA8000324F3E798B108B503460020C3F8B802E8
:107BB800C3F8C402C3F8D00209B1C3F8B412012152
:107BC80083F89C121A70184600F0F0FF08BD0320D5
:107BD800704710B582B00023ADF8063089B104466D
:107BE800C0F8B812CB6A23B10DF106009847C4F863
:107BF800D002D4F8D8320133C4F8D832002002B009
:107C080010BD0320FBE708B501F033F808BD08B53F
:107C1800D0F8B83213B11B68984708BD0020FCE7BC
:107C280008B5D0F8B8325B68984700B908BD03209A
:107C3800FCE738B5044600F2AA25284600F0C9F941
:107C48000123C4F89432B4F8B032C4F8983294F8E6
:107C5800AA1201F01F03012B0DD0022B10D02BB15B
:107C680001F08001204601F01FF803E02946204674
:107C780000F084FB38BD2946204600F0BAFBF9E73E
:107C88002946204600F0F7FBF4E7F8B5044601233F
:107C980080F89C320023C0F894324360C0F8A432C4
:107CA80080F8A032D0F8B832DBB15B68DBB10021D4
:107CB80098470746C8B9402300221146204600F0DD
:107CC800E0FF0126A4F864614025C4F860512B4602
:107CD80000228021204600F0D4FFA6842562384681
:107CE800F8BD0027E7E70027E5E70327E3E7017486
:107CF8000020704790F89C32DBB2042B04D090F837
:107D08009C32DBB280F89D32042380F89C3200203C
:107D1800704790F89C32DBB2042B01D000207047EA
:107D280090F89D32DBB280F89C32F7E708B590F8FE
:107D38009C32DBB2032B01D0002008BDD0F8B8324A
:107D4800002BF9D0DB69002BF6D09847F4E708B58B
:107D5800D0F8D432AE3350F823205AB190F89C3280
:107D6800DBB2032B01D0002008BD136A23B198476A
:107D78000020F9E70320F7E70020F5E708B5D0F879
:107D8800D432AE3350F823205AB190F89C32DBB28B
:107D9800032B01D0002008BD536A23B19847002067
:107DA800F9E70320F7E70020F5E70020704708B55A
:107DB800012380F89C32D0F8B83223B15B6801798E
:107DC800984710B908BD0020FCE70320FAE7002017
:107DD80070470020704738B504460D46002943D146
:107DE8001346D0F89422032A01D0084638BDD0F8AB
:107DF8005C11D0F86021914212D890F8AA3203F0B1
:107E08001F03012B17D0022B1CD0284694F89C3254
:107E1800DBB2032B1BD0204600F095FC2846E5E793
:107E2800891AC0F85C118A4228BF0A46194600F030
:107E380082FC2846DAE790F8AE12FFF7C8FF002860
:107E4800E9D1E3E790F8AE12FFF7C3FFF7E700F1D7
:107E5800AE0354F823301A69002ADCD0C4F8D402DF
:107E68001B6920469847D6E701F07F01FFF7B1FF6D
:107E780090B994F89C32DBB2032BB7D100F1AE0372
:107E880054F823309A69002AB0D0C4F8D4029B6908
:107E9800294620469847A9E70020A7E738B50446B1
:107EA8000D4600294BD11346D0F89422022A07D058
:107EB80094F8A00218B1002384F8A032284638BDEF
:107EC800C269016A8A420ED88A4218D094F89C3254
:107ED800DBB2032B27D08021204600F0E5FE2046A8
:107EE80000F03CFCE4E7521AC261194600F00CFCB1
:107EF80000231A461946204600F0F6FED8E78369A3
:107F08009942E3D8D0F898229342DFD20022114652
:107F180000F0FAFB0021C4F898120B460A462046E6
:107F280000F0E2FEC4E7D4F8B832DA68002AD2D00A
:107F38000022C4F8D422DB6820469847CBE741F0FA
:107F48008001FFF746FF90B994F89C32DBB2032B0F
:107F5800B5D100F1AE0354F823305A69002AAED0E7
:107F6800C4F8D4025B69294620469847A7E7002051
:107F7800A5E703780A8813440B80037818447047F0
:107F8800428803789A4218D930B583B004460D4622
:107F9800ADF806306288BDF806309A420AD90DF16C
:107FA8000601FFF7E6FF4378052BF3D18378AB4250
:107FB800F0D100E0002003B030BD00207047034638
:107FC800002002E00130C0B201331A78002AF9D14A
:107FD80070470B7803704B7843708B78CA7843EA04
:107FE800022343800B794A7943EA022383808B7901
:107FF800CA7943EA0223C380704710B5044680213A
:1080080000F052FE0021204600F04EFE10BD30B5B3
:1080180083B004460D460023ADF806304A88130A9B
:10802800013B062B00F2AB80DFE803F0041F33A905
:10803800A98D9A00D0F8B4321B680DF10601007CB6
:108048009847EA88002A00F0A380BDF80630002B84
:1080580000F099809A4228BF1A46ADF806200146DA
:10806800204600F044FB03B030BD037C43B9D0F890
:10807800B8329B6A0DF10600984702234370E0E787
:10808800D0F8B832DB6A0DF1060098470223437036
:10809800D7E7D2B2052A52D8DFE802F003101D2A2A
:1080A8003744D0F8B4325B6823B10DF10601007C87
:1080B8009847C6E72946FFF7A0FFD4E7D0F8B432BF
:1080C8009B6823B10DF10601007C9847B9E7294662
:1080D800FFF793FFC7E7D0F8B432DB6823B10DF19F
:1080E8000601007C9847ACE72946FFF786FFBAE708
:1080F800D0F8B4321B6923B10DF10601007C984712
:108108009FE72946FFF779FFADE7D0F8B4325B69FE
:1081180023B10DF10601007C984792E72946FFF745
:108128006CFFA0E7D0F8B4329B6923B10DF10601CA
:10813800007C984785E72946FFF75FFF93E72946C4
:10814800FFF75BFF8FE7037C33B9D0F8B8325B6B7E
:108158000DF10600984774E72946FFF74EFF82E7BE
:10816800037C43B9D0F8B8321B6B0DF10600984771
:108178000723437065E72946FFF73FFF73E7294662
:10818800FFF73BFF6FE729462046FFF736FF6AE710
:10819800204600F0D8FA66E738B504468B88FBB964
:1081A800CB88EBB94B887F2B1AD803F07F0590F862
:1081B8009C32DBB2032B0CD080F89E52294600F08B
:1081C80083FD204600F0BFFA35B1022384F89C32C3
:1081D80009E0FFF712FF06E0012384F89C3202E071
:1081E8002046FFF70AFF38BD70B504460E468D7865
:1081F8002F4B1D70012D10D890F89C32DBB2022B4A
:108208000FD0032B26D0FFF7F8FE294B197820460C
:10821800FFF706FD0325284670BDFFF7EEFE032590
:10822800F9E7A5B145602946FFF7F1FC054638B1E5
:1082380031462046FFF7E1FE022384F89C32EAE744
:10824800204600F080FA032384F89C32E3E700F02C
:108258007AFAE0E7CDB141688D4225D0C9B2FFF77F
:10826800DFFC134B197861602046FFF7D0FC054608
:10827800B0B131462046FFF7C0FE21792046FFF70E
:10828800CFFC022384F89C32C5E7022380F89C3295
:1082980045602946FFF7C4FC204600F054FABAE7C7
:1082A800204600F050FAB6E700F04DFA0025B2E794
:1082B800B80E002408B5CB88012B0BD190F89C325E
:1082C800DBB2022B09D9032B09D10122011D00F0D1
:1082D8000EFA01E0FFF791FE08BD5BB213B9FFF794
:1082E8008CFEF9E70146002341F8083F012200F01F
:1082F800FEF9F1E708B590F89C32013B022B12D841
:10830800CB88022B0CD10123C360D0F8A4320BB167
:108318000323C360022200F10C0100F0E8F908BD54
:10832800FFF76BFEFBE7FFF768FEF8E708B54B8839
:10833800012B04D0022B07D0FFF75FFE08BDC0F861
:10834800A43200F000FAF9E78B881B0A80F8A03203
:1083580000F0F9F9F2E708B590F89C32013B022BDE
:1083680009D84B88012B00D008BD0023C0F8A432DF
:1083780000F0E9F9F8E7FFF740FEF5E738B50C78C3
:1083880004F06004202C06D0402C04D06CB1FFF718
:1083980034FE002407E0D0F8D432AE3350F823304E
:1083A8009B6898470446204638BD4D78092D1DD84E
:1083B800DFE805F012191C161C08051C0F0BFFF747
:1083C80026FEF0E7FFF7E8FEEDE7FFF70DFF0446AE
:1083D800E9E7FFF76FFFE6E7FFF78CFF2C46E2E7D8
:1083E800FFF7A4FFDFE7FFF7B6FFDCE7FFF705FEBF
:1083F800D9E770B505460C460B7803F06003202BCF
:1084080007D0402B05D023B1FFF7F7FD00263046F3
:1084180070BD95F89C32013B022B26D821790129A1
:1084280005D921462846FFF7E8FD0026EFE728464C
:10843800FFF7CDFC68B900F1AE0255F8222091682B
:1084480089B1C5F8D402936821462846984706465C
:1084580000E00326E388002BD9D1002ED7D1284687
:1084680000F071F9D3E70326F4E721462846FFF721
:10847800C4FD0026CBE72DE9F04106460D468B8862
:10848800DFB20C7804F06004202C08D0402C06D011
:10849800DCB1FFF7B2FD00242046BDE8F081394683
:1084A8003046FFF796FC0446002840F0F980C6F8ED
:1084B800D40200F1AE0356F823309B68002BEBD0B2
:1084C8002946304698470446E6E791F80180B8F116
:1084D800010F31D0B8F1030F05D0B8F1000F66D005
:1084E800FFF78BFDD8E790F89C32DBB2022B04D063
:1084F800032B11D0FFF781FDCEE7002F18BF802F87
:1085080007D0394600F0D0FB8021304600F0CCFB84
:10851800C2E7FFF772FDBFE74B882BB9002F18BFE2
:10852800802F01D0CB881BB1304600F00CF9B3E79F
:10853800394600F0B9FBF7E790F89C32DBB2022B22
:1085480004D0032B11D0FFF758FDA5E7002F18BF63
:10855800802F07D0394600F0A7FB8021304600F075
:10856800A3FB99E7FFF749FD96E74B88002B93D1CA
:1085780017F07F0F17D1304600F0E5F8394630463E
:10858800FFF727FC002887D1C6F8D40200F1AE0215
:1085980056F822209268002A00F084802946304646
:1085A8009047044678E7394600F086FBE3E790F801
:1085B8009C22D2B2022A05D0032A28D0FFF71DFD3B
:1085C800444669E7002F18BF802F13D113F0800F9E
:1085D80014D107F07F0707EB8707B90001F5A871E9
:1085E8000144043100230B600222304600F07FF87A
:1085F800444651E7FFF701FD44464DE707F07F0782
:1086080007EB8707B900103101440431EAE75BB290
:10861800002B20DB07F00F0202EB820200EB820244
:10862800B2F8642122B3002B26DB07F07F0303EBAB
:1086380083039C0004F5A87434440434802F18BFC5
:10864800002F22D10023236002222146304600F069
:108658004EF8444620E707F00F0202EB820200EBD7
:108668008202928C002ADED1FFF7C7FC444613E74A
:10867800FFF7C3FC44460FE707F07F0303EB8303D0
:108688009C00103434440434D8E73946304600F0AE
:10869800C5FA10B101232360D6E700232360D3E78E
:1086A8000024F9E60446F7E600B370B50D46164611
:1086B8000446FFF784FC01304300B3F5007F06D879
:1086C8009BB233802B7003236B7002230AE04FF4B4
:1086D8000073F6E7EA5401345A1CD2B20021A954B7
:1086E8000233DBB22278002AF4D170BD704708B596
:1086F80013460222C0F894228361C3610A4600210E
:1087080000F0EAFA002008BD08B513460A46002121
:1087180000F0E2FA002008BD08B513460322C0F8AD
:108728009422C0F85831C0F85C310A46002100F0A4
:10873800DBFA002008BD08B513460A46002100F000
:10874800D3FA002008BD08B50422C0F894220023FB
:108758001A46194600F0C0FA002008BD08B50522DF
:10876800C0F8942200231A46194600F0BDFA0020EA
:1087780008BD000008B5012210491148FFF712FA98
:1087880080B910490E48FFF724FA70B90E490C4811
:10879800FFF7AAF960B90A48FFF735FA58B9FBF7A5
:1087A800BDF808BDF8F78AFAEBE7F8F787FAEDE7BE
:1087B800F8F784FAEFE7F8F781FAF0E7AC0000245D
:1087C800BC0E0024100000249800002400207047EC
:1087D800002070470020704710B50146044C204621
:1087E800FFF79BF92046FFF7C1F9002010BD00BF35
:1087F800BC0E002410B5064C002206492046FFF79F
:108808007EF905492046FFF788F9002010BD00BF12
:10881800BC0E00249819002498110024094BD3F8A1
:10882800BC32D3F814320BB10120704710B5054C97
:108838000A4601462046FFF762F92046FFF779F914
:1088480010BD00BFBC0E002412230B8000487047E7
:10885800C800002404230B8000487047DC00002473
:10886800002393421ED200B510E00CF1370C01F83A
:1088780013C000014FEA430C0CF1010C4FF0000E3D
:1088880001F80CE00133DBB2934209D24FEA107CC5
:10889800B0F1204FE9D20CF1300C01F813C0E8E731
:1088A8005DF804FB7047000038B50B4BD3F800089F
:1088B800D3F80448D3F80838C01800D138BD074D9C
:1088C8000822A91CFFF7CCFF042205F1120120465B
:1088D800FFF7C6FFF2E700BF00E0F11FE000002449
:1088E80008B51A230B80FFF7DFFF014808BD00BF5A
:1088F800E000002408B50A4628B905490548FFF7ED
:10890800D3FE034808BD02490248FFF7CDFEF8E749
:1089180098210024C09E000810B50A46034C214641
:108928000348FFF7C1FE204610BD00BF9821002470
:10893800D89E000808B50A4628B905490548FFF732
:10894800B3FE034808BD02490248FFF7ADFEF8E749
:1089580098210024EC9E000808B50A4628B9054964
:108968000548FFF7A1FE034808BD02490248FFF782
:108978009BFEF8E798210024F89E0008F0B5BDB0EA
:10898800044600213791389139913A913B91C022A0
:1089980006A800F0DBF92268474B9A4201D03DB0A7
:1089A800F0BD4FF480220023CDE906234FF4401395
:1089B800289306A8FBF7BCFE002879D1FAF7AEFF8A
:1089C8003E4CD4F8E03043F00403C4F8E030D4F867
:1089D800E03003F004030193019BD4F8E03043F046
:1089E8000103C4F8E030D4F8E03003F00103029347
:1089F800029BD4F8E03043F00203C4F8E030D4F826
:108A0800E03003F002030393039B0D233793022600
:108A18003896002539953A960A273B9737A928486A
:108A2800F9F7C2FF28233793389639953A963B973A
:108A380037A92448F9F7B8FF43F623433793389604
:108A480039953A963B9737A91F48F9F7ADFFD4F8FF
:108A5800D83043F00073C4F8D830D4F8D83003F0D5
:108A680000730493049BD4F8D83043F08063C4F8AF
:108A7800D830D4F8D83003F080630593059B2A4694
:108A880029464A20F8F75CFD4A20F8F78FFD2A4668
:108A980029464B20F8F754FD4B20F8F787FD2A4666
:108AA80029464D20F8F74CFD4D20F8F77FFD76E775
:108AB800F8F704F982E700BF0000044000440258B8
:108AC80000080258000002580004025808B500F2D5
:108AD8009C41D0F8E004FFF7ACF808BD08B501EBFD
:108AE800C10300EB8303D3F86022D0F8E004FFF75A
:108AF80072F908BD08B501EBC10300EB83031A6ADC
:108B0800D0F8E004FFF7CAF908BD08B5D0F8E004CA
:108B1800FFF70CF908BD10B50446C17911B1022957
:108B280009D10121D4F8E004FFF7E1F8D4F8E00412
:108B3800FFF7ABF810BDF8F7C1F80121F2E7000024
:108B480010B50446D0F8E004FFF7D4F82268D2F84C
:108B5800003E43F00103C2F8003EE37A23B1034A22
:108B6800136943F00603136110BD00BF00ED00E078
:108B780008B5D0F8E004FFF7CCF808BD08B5D0F880
:108B8800E004FFF7FBF808BD08B5D0F8E004FFF7EC
:108B9800DEF808BD08B5D0F8E004FFF706F908BD0F
:108BA80008B5D0F8E004FFF702F908BD0378012BF7
:108BB80001D00020704710B5164BC3F8E004C0F888
:108BC800C832154A1A6009221A710022DA719A719C
:108BD800012159729A72DA721A739A73DA731A74D3
:108BE8001846FAF76CF890B90A4C4FF40071204611
:108BF800FAF74FFE802200212046FAF725FE4FF4AF
:108C0800BA7201212046FAF71FFE002010BDF8F7BE
:108C180055F8E9E79823002400000440D0F8C8324A
:108C280011F0800F08D101F07F0101EBC10103EBC6
:108C3800810191F85602704701F07F0101EBC101F3
:108C480003EB8101887D704708B5D0F8C802FAF7B0
:108C580037FA08BD004870477C280024704703286D
:108C680005D8DFE800F0050402050120704703205D
:108C7800704708B5D0F8C802FAF7A2F8FFF7EFFF77
:108C880008BD08B594461A466346D0F8C802FAF7F4
:108C980076F9FFF7E4FF08BD08B5D0F8C802FAF77F
:108CA800B2F9FFF7DCFF08BD08B5D0F8C802FAF73B
:108CB80035FAFFF7D4FF08BD08B5D0F8C802FAF7AF
:108CC80070FAFFF7CCFF08BD08B5D0F8C802FAF76C
:108CD80043F9FFF7C4FF08BD08B5D0F8C802FAF792
:108CE800F8F9FFF7BCFF08BD08B5D0F8C802FAF7D5
:108CF800C2F9FFF7B4FF08BD014B1868704700BF01
:108D0800FC00002470B50D4E0D4D761BB61006D034
:108D1800002455F8043B01349847A642F9D1094E7E
:108D2800094D761B01F09CF8B61006D0002455F8C2
:108D3800043B01349847A642F9D170BD149F00083E
:108D4800149F00081C9F0008149F0008830730B573
:108D580048D0541E002A3FD0CAB2034601E0013C65
:108D68003AD303F8012B9D07F9D1032C2DD9CDB2A5
:108D780045EA05250F2C45EA054536D9A4F1100228
:108D880022F00F0C03F1200EE6444FEA121C03F107
:108D9800100242E9045542E9025510327245F8D1F1
:108DA8000CF1010214F00C0F03EB021204F00F0C8B
:108DB80013D0ACF1040323F003030433134442F843
:108DC800045B9342FBD10CF003042CB1CAB21C44DF
:108DD80003F8012B9C42FBD130BD64461346002C9E
:108DE800F4D1F9E703461446BFE71A46A446E0E77C
:108DF8002DE9F043694CD4F8008083B004460E4650
:108E080017461D46B8F1000F03D0D8F83830002BAC
:108E180077D0022F05D0012F00F2AC80002DC0F2D0
:108E2800A980636EDA0752D52146404600F058F90A
:108E3800216B41B104F14003994202D0404600F051
:108E48007BFA00232363B4F90CC000231CF0800FC5
:108E5800A361636064D12CF44A6C2CF0030C022FDC
:108E6800A4F80CC06AD001AB6A462146404600F01F
:108E780095FBA3891843A081002D2FD0002E2ED05A
:108E8800D8F83830002B38D0009B2660AB42B4F9B4
:108E98000C301CBF43F40063A381012F04BF43F0CF
:108EA8000103A3819AB213F00803C4E904652CD026
:108EB800D1075DD56D42A561656E002315F00105EA
:108EC800A36027D00025284603B0BDE8F083A38916
:108ED8009B05A9D4A06D00F05DFBA5E7009D284681
:108EE80000F08CFB0646002847D0A38943F0800396
:108EF800A381D8F83830002BC6D1404600F024F9B9
:108F0800C2E7404600F020F983E7A360656E15F0DC
:108F18000105D7D1930524D5284603B0BDE8F083D1
:108F28002169404600F008FAB4F90CC02CF44A6CE8
:108F38002CF0030C022FA4F80CC094D100250022B9
:108F480004F14303A2600122C4E904322360636E82
:108F58004CF0020CD807A4F80CC0DDD41CF4007F38
:108F6800DAD1A06D00F018FB284603B0BDE8F08305
:108F7800A560CBE74FF0FF35CEE7DDF80090A945B7
:108F880004D0484600F03AFB064620B9B4F90CC0B4
:108F98004FF0FF35D3E74D46A7E700BFFC0000249C
:108FA800024B13B1024800F005B8704700000000FA
:108FB80075920008002301461A46184600F050BE74
:108FC800B1F90C20F8B50C461107074642D463687E
:108FD80042F40062002BA28159DDA56A002D54D00D
:108FE80000233E683B6093B212F4805253D1E1698A
:108FF80001233846A847421C63D0A389A56A5B07AA
:1090080005D56368C01A236B0BB1E36BC01AE1691D
:10901800024600233846A847411C3ED13B68002B36
:109028003BD01D2B01D0162B52D1A3892269226077
:1090380023F4006300216160A381216B3E6021B3AA
:1090480004F14003994202D0384600F075F9002037
:109058002063F8BD2669C6B193B2256826609A07D1
:109068000CBF63690023AD1BA3600CE0D4F824C0D7
:10907800E1692B4632463846E047B0F1000CA5EBD3
:109088000C05664416DD002DF0DC0020F8BDE36B0E
:10909800002BA2DCF9E7206DB1E7B4F90C302269A6
:1090A800226023F40063A3810022DB046260C4D53C
:1090B8002065C2E7A38943F040034FF0FF30A38146
:1090C800F8BD3B68002B98D01D2B06D0162B04D07A
:1090D800A38943F04003A381F8BD3E60D5E700BFF4
:1090E80038B50C46054608B1836BA3B1B4F90C003A
:1090F800B8B1636EDB0701D4810515D52846214632
:10910800FFF75EFF636EDA07054602D4A3899B0565
:109118000ED5284638BD00F017F8B4F90C00002821
:10912800E7D10546284638BDA06D00F033FAE5E7DB
:10913800A06D00F031FA284638BD00BF014900F0A3
:1091480001BA00BF199D00082DE9F0478246394849
:1091580000F020FADAF83840002C66D1DAF804502A
:10916800354ACAF83C200323CAE9B843DFF8CC9053
:10917800DFF8CC80334F344E04230AF53B72CAF82B
:10918800E8222146C5E90243C5E90044C5E904448B
:109198006C660822AC6105F15C00FFF7D7FDC5E9F4
:1091A8000759C5E90987EE6205F1580000F0EEF9A4
:1091B800DAF80850254BEB602146C5E90044C5E9BB
:1091C80004446C66AC60AC61082205F15C00FFF7F2
:1091D800BDFDC5E90759C5E90987EE6205F15800E3
:1091E80000F0D4F9DAF80C50194BEB602146C5E9C8
:1091F8000044C5E904446C66AC60AC61082205F122
:109208005C00FFF7A3FD05F15800C5E90759C5E95A
:109218000A76C5F8248000F0B9F90123CAF8383075
:109228000448BDE8F04700F0B7B9BDE8F047014889
:1092380000F0B2B9A82A002445910008B19B0008A3
:10924800D59B0008159C0008359C00080900010002
:1092580012000200014800F09DB900BFA42A0024B2
:10926800014800F099B900BFA42A002438B5084B7A
:10927800084D5B1B9C1007D0043B1D44013C55F86E
:1092880004399847002CF9D1BDE8384000F0EEBD0C
:10929800209F00081C9F0008F8B5244F0C4606467E
:1092A80000F064FCBA685568C4F57E630F3325F096
:1092B80003052B4423F47F6323F00F03A3F58054A5
:1092C800B4F5805F07DB0021304600F05BFCBB682B
:1092D8002B44984204D0304600F04EFC0020F8BDE4
:1092E8006142304600F04EFC01300DD0104ABB6898
:1092F8002D1B45F001055D60136830461B1B13608C
:1093080000F03AFC0120F8BD0021304600F03AFC9C
:10931800BA68831A0F2BDEDD43F001035360054B57
:1093280003491B68C01A0860D5E700BF2C05002454
:10933800AC2A002434090024002961D0F8B50C4671
:10934800064600F013FC54F8042C7B4FA4F10805E2
:1093580022F0010105EB010CB868DCF80430604527
:1093680023F0030300F08B80D207CCF8043032D40A
:1093780054F8082CAD1A1144AA6807F10800824273
:109388006AD00CEB0304D4F804E0EC68D4601EF057
:10939800010FA26000F0978041F001036B60CCF8E8
:1093A8000010B1F5007F35D27A68CB084809012151
:1093B800013381401143796007EBC30257F833103A
:1093C800083AC5E9021247F83350CD603046BDE887
:1093D800F84000F0D1BB0CEB03025268D00710D460
:1093E800194407F10800DCF80830834273D0DCF830
:1093F8000C20DA60936041F001036B606950D0E79C
:10940800704741F00103B1F5007F44F8043CCCF803
:109418000010C9D3B1F5206F4FEA512348D28B0908
:1094280003F1390003F13802C300F818FB58083873
:10943800984259D05A6822F003028A4202D99B689E
:109448009842F7D1D868C5E902308560DD603046BA
:10945800BDE8F84000F090BB0CEB03025268D2075D
:1094680063D40B44DCE90212CA60916043F0010244
:109478006A603046EB50BDE8F84000F07DBB0B4415
:10948800D10707D454F8082CAD1A1344D5E90212B1
:10949800CA60916043F001026A60284ABD601268A0
:1094A8009A4293D8264B30461968FFF7F5FE8DE7A8
:1094B800142B0AD9542B1FD80B0B03F16F0003F19F
:1094C8006E02C300B1E719448DE703F15C0003F1B4
:1094D8005B02C300A9E741F00103C7E90455C5E9E8
:1094E80002006B60695071E779689210012404FAF0
:1094F80002F20A437A60A6E7B3F5AA7F06D8CB0B37
:1095080003F1780003F17702C3008EE740F254526A
:10951800934206D88B0C03F17D0003F17C02C30053
:1095280083E74FF47E737E227FE741F001036B608F
:10953800CCF800104AE700BF2C05002438090024A5
:10954800DC2A00242DE9F8430746884600F53876DA
:109558004FF00009D6E90154013D11D4A389012B2C
:1095680005F1FF3508D9B4F90E300133214603D08F
:109578003846C04749EA00096B1C04F16804EDD17C
:109588003668002EE6D14846BDE8F883704700BF2C
:10959800704700BF704700BF704700BF70B50C46EA
:1095A800B1F90E10002996B015461E4614DB6A461E
:1095B80000F014FC00280FDB019A02F47042A2F5B7
:1095C8000052B2FA82F24FF4806352094FF40060FD
:1095D80032602B6016B070BDB4F90C10002311F086
:1095E8008000336004D0402218462A6016B070BD4F
:1095F8004FF480632B6016B070BD00BF024B01466C
:10960800186800F003B800BFFC0000242DE9F04FF3
:1096180001F10B06162E83B0044624D8102900F257
:10962800BA8000F0A3FA102618220220B54F3A4457
:10963800A2F1080153688B4200F0BA805A68D968D1
:1096480022F003021A449D68E9608D60516841F078
:1096580001012046516003F1080500F08DFA284603
:1096680003B0BDE8F08F36F0070600F19480B142F0
:1096780000F2918000F07AFAB6F5FC7FC0F09A818A
:10968800730A00F08F80042B00F26F81B30903F195
:10969800390003F1380CC3009A4F3B44A3F1080585
:1096A8005B689D4206D10CE0002980F22781DB68C7
:1096B8009D4206D05A6822F00302911B0F29F3DD60
:1096C80060463D69DFF840C265457CD06A6822F093
:1096D8000302931B0F2B00F37B81002BC7E904CCFB
:1096E80080F26C81B2F5007F80F01A81D308796826
:1096F80001334FEA521E012202FA0EF20A4357F8CA
:1097080033E0C5F808E007EBC3010839E9607A607F
:1097180047F83350CEF80C508310012199409142FC
:1097280057D8114206D120F003004900114200F138
:109738000400FAD007EBC0094D468646D5F80C80E0
:10974800454508D11DE1002B80F22481D8F80C8012
:10975800454500F01681D8F8042022F00302931B37
:109768000F2BF0DD2046D8E9025408EB060146F03D
:109778000106C8F80460EC60A56043F00104C7E97D
:109788000411C1E902CC4C6048F8023000F0F4F949
:1097980008F1080502E00C2323600025284603B0E1
:1097A800BDE8F08F4FF4007340204FF03F0C73E793
:1097B800D3689A4208BF02307FF440AF3D69DFF8B2
:1097C80048C1654582D17A68831001219940914248
:1097D800A7D9BD686B6823F003094E4503D8A9EBE8
:1097E80006030F2B7ADCDFF824B1494BDBF80020A5
:1097F8001B680132334405EB090A00F0338103F595
:1098080080530F3323F47F6828F00F084146204621
:1098180000F0B8F9411C024600F0F380824500F2DE
:10982800EE803C4B196841441960084600F04E81AF
:10983800DBF80010019301311BBFA2EB0A0A504468
:10984800CBF80020186012F0070B00F01781CBF15D
:1098580008010A44CBF5805190440831A1EB080176
:10986800C1F30B0A51462046009200F08BF9421CC6
:10987800DDE9002300F04F81801A00EB0A0819681F
:10988800BA6048F001005144BD425060196000F0D0
:109898002981B9F10F0F40F227816868A9F10C0CF2
:1098A8002CF0070C00F0010040EA0C0068604FF053
:1098B800050E05EB0C00BCF10F0FC0E901EE00F23C
:1098C800328150681546144B1A688A4238BF1960AD
:1098D800124B1A688A4238BF196094E0AA1943F0FB
:1098E800010346F001066E602046BA60536000F03E
:1098F80043F90835284603B0BDE8F08FD9681A4403
:10990800A1E600BF2C0500243405002434090024F6
:10991800DC2A0024AC2A0024D42A0024D82A0024D3
:10992800B2F5206F4FEA522363D3142B00F2B780AD
:1099380003F15C01C9005B3307EB010E7958AEF106
:10994800080E8E4500F091804B6823F00303934284
:1099580002D989688E45F7D1D1F80CE07A68C5E953
:10996800021ECEF80850CD60D6E6142B59D9542BD8
:1099780000F29D80330B03F16F0003F16E0CC300FE
:109988008AE60EF1010E1EF0030F05F108057FF4BB
:10999800D5AE51E0424445465368D8F80C1043F020
:1099A8000103536055F8083F2046D9608B6000F0EA
:1099B800E3F8F3E6F00806F1080237E62A44204601
:1099C800536843F001035360083500F0D5F8E5E625
:1099D800A919204646F0010643F001046E60C7E964
:1099E8000411C1E902CC4C60AB5000F0C5F8083551
:1099F800D4E6930903F13901C90038339CE7BD4225
:109A08005FD0BD68686820F003084645A8EB0603E8
:109A180002D80F2B3FF762AF204600F0ADF80025C3
:109A2800BCE603F15C0003F15B0CC30034E659F8B3
:109A380008394B4540F0968010F0030F00F1FF30D5
:109A4800F5D17B6823EA01037B60490099423FF620
:109A5800C0AE19B9BDE649000EF1040E1942FAD09C
:109A6800704667E603F11008D0E69A104FF0010837
:109A78007B6808FA02F21A437A6070E702EB080181
:109A88004942C1F30B0A51462046009200F07AF889
:109A9800431CDDE900237FF4EFAEDA46EFE6542BF2
:109AA80025D8130B03F16F01C9006E3344E7B3F5F2
:109AB800AA7F25D8F30B03F1780003F1770CC300D4
:109AC800EAE5294B186840441860B1E6CAF30B0C64
:109AD800BCF1000F7FF4ACAEBD68C84448F001008B
:109AE8006860F0E61546EEE60123536094E7B3F5A7
:109AF800AA7F23D8D30B03F17801C90077331BE77A
:109B080040F25452934223D8B30C03F17D0003F181
:109B18007C0CC300C0E5ABF1080BD844A8EB0208E5
:109B28004FF0000AABE605F1080120460093FFF765
:109B380003FCBD68009B68681968C4E640F254518C
:109B48008B420BD8930C03F17D01C9007C33F3E6FB
:109B58004FF47E737F204FF07E0C9DE54FF47E71AD
:109B68007E23E9E67B6870E7AC2A00240148FFF70A
:109B780011BD00BFA02A00240148FFF70DBD00BF9A
:109B8800A02A002438B5074D0022044608462A605A
:109B9800F7F778FA431C00D038BD2B68002BFBD0B0
:109BA800236038BDE02A002410B50C46B1F90E1028
:109BB80000F040F9002803DB236D0344236510BD42
:109BC800A38923F48053A38110BD00BF2DE9F04180
:109BD8000C46B1F90C101F46CB05054616460BD4AA
:109BE80021F48051A1813B46B4F90E103246284633
:109BF800BDE8F04100F01EB8B4F90E1002230022AF
:109C080000F002F9B4F90C10EAE700BF10B50C46F1
:109C1800B1F90E1000F0F8F8A389421C0EBF23F426
:109C2800805343F480532065A38110BDB1F90E1011
:109C380000F05CB838B50C46084D844611462046FD
:109C48001A4600232B606446F7F768F9431C00D0D6
:109C580038BD2B68002BFBD0236038BDE02A0024D8
:109C68002DE9F047DFF87CA00646DAF800009846B0
:109C78000F469146FFF78EFC1B4B1B68D3F84841F3
:109C880024B365681F2D26DC5EB96B1C0235DAF833
:109C98000000636044F82570FFF77EFC0020BDE8F3
:109CA800F08704EB85010123C1F88890D4F8882156
:109CB800AB401A43022EC4F88821C1F80881E4D1C8
:109CC800D4F88C211343C4F88C31DEE703F5A6746D
:109CD800C3F84841D5E7DAF80000FFF75DFC4FF01C
:109CE800FF30DCE728050024089F000838B5074D39
:109CF8000022044608462A60F7F72AF9431C00D0D8
:109D080038BD2B68002BFBD0236038BDE02A002427
:109D180070B500294BD006460C4610B1836B002B5A
:109D280048D0636ED80734D5B4F90C30002B3ED038
:109D380021463046FFF744F9E36A054633B1E16945
:109D4800304698470028B8BF4FF0FF35A3891A0658
:109D58003BD4216B41B104F14003994202D0304613
:109D6800FFF7EAFA00232363616C21B13046FFF75D
:109D7800E3FA00236364FFF76DFA636E0022DB07E2
:109D8800A28127D5A06DFFF703FCFFF769FA2846E3
:109D980070BDA3899905CBD4A06DFFF7FBFBB4F97F
:109DA8000C30002BC4D1656E15F0010508D00025D4
:109DB800284670BDFFF7C8F9636ED807B4D4E8E742
:109DC800A06DFFF7E9FB284670BD21693046FFF713
:109DD800B3FABEE7A06DFFF7DFFBD3E770B50C461B
:109DE800084D03460026204611461C462E60F7F70C
:109DF800DBF8431C00D070BD2B68002BFBD0236020
:109E080070BD00BFE02A002438B50C46084D8446D2
:109E1800114620461A4600232B606446F7F7A4F83B
:109E2800431C00D038BD2B68002BFBD0236038BD05
:109E3800E02A002438B50C46084D844611462046D1
:109E48001A4600232B606446F7F796F8431C00D0A7
:109E580038BD2B68002BFBD0236038BDE02A0024D6
:109E6800F8B500BFF8BC08BC9E467047F8B500BFFF
:089E7800F8BC08BC9E467047CF
:109E800000000000010203040102030406070809A0
:109E9000000610160006101601000200040006005D
:109EA00008000A000C0010002000400080000001A3
:109EB0000804020408010101010101030701000077
:109EC00053544D3332205669727475616C20436F60
:109ED0006D506F727400000053544D6963726F656A
:109EE0006C656374726F6E69637300004344432052
:109EF000436F6E666967000043444320496E746592
:0C9F00007266616365000000000100242F
:089F0C00F868FF7F010000006E
:089F1400A98F0008BD0200083E
:049F1C00990200089E
:109F20000090D0030090D00301000000100000005A
:109F3000037A00089F790008857800080000000077
:109F4000AD76000809780008D1770008000000000D
:109F50000000000000000000897700084177000839
:109F6000F9760008ED76000809024300020100C0FE
:109F7000320904000001020201000524001001055D
:109F800024010001042402020524060001070582C1
:109F90000308001009040100020A0000000705017F
:109FA0000240000007058102400000000A0600028E
:109FB0000000004001000000FD870008D587000870
:109FC000D9870008E1870008DD870008518800086C
:109FD0005D88000821890008FD880008E9880008DC
:109FE0003D89000861890008120100020202004058
:109FF0008304405700020102030100000403090426
:10A000001A03000000000000000000000000000033
:10A01000000000000000000000000000000100241B
:10A0200000000000EC03002454040024BC040024BD
:10A030000000000000000000000000000000000020
:10A040000000000000000000000000000000000010
:10A050000000000000000000000000000000000000
:10A0600000000000000000000000000000000000F0
:10A0700000000000000000000000000000000000E0
:10A0800000000000000000000000000000000000D0
:10A0900000000000000000000000000000000000C0
:10A0A00000000000000000000000000000000000B0
:10A0B00000000000000000000000000000000000A0
:10A0C000000000000000000001000000000000008F
:10A0D0000E33CDAB34126DE6ECDE05000B00000054
:10A0E0000000000000000000000000000000000070
:10A0F0000000000000000000000000000000000060
:10A10000000000000000000000000000000000004F
:10A11000000000000000000000000000000000003F
:10A4400000000000000000009C2A00240000000022
:10A45000000000002C0500242C05002434050024F5
:10A46000340500243C0500243C0500244405002458
:10A47000440500244C0500244C0500245405002408
:10A48000540500245C0500245C05002464050024B8
:10A49000640500246C0500246C0500247405002468
:10A4A000740500247C0500247C0500248405002418
:10A4B000840500248C0500248C05002494050024C8
:10A4C000940500249C0500249C050024A405002478
:10A4D000A4050024AC050024AC050024B405002428
:10A4E000B4050024BC050024BC050024C4050024D8
:10A4F000C4050024CC050024CC050024D405002488
:10A50000D4050024DC050024DC050024E405002437
:10A51000E4050024EC050024EC050024F4050024E7
:10A52000F4050024FC050024FC0500240406002496
:10A53000040600240C0600240C0600241406002443
:10A54000140600241C0600241C06002424060024F3
:10A55000240600242C0600242C06002434060024A3
:10A56000340600243C0600243C0600244406002453
:10A57000440600244C0600244C0600245406002403
:10A58000540600245C0600245C06002464060024B3
:10A59000640600246C0600246C0600247406002463
:10A5A000740600247C0600247C0600248406002413
:10A5B000840600248C0600248C06002494060024C3
:10A5C000940600249C0600249C060024A406002473
:10A5D000A4060024AC060024AC060024B406002423
:10A5E000B4060024BC060024BC060024C4060024D3
:10A5F000C4060024CC060024CC060024D406002483
:10A60000D4060024DC060024DC060024E406002432
:10A61000E4060024EC060024EC060024F4060024E2
:10A62000F4060024FC060024FC0600240407002491
:10A63000040700240C0700240C070024140700243E
:10A64000140700241C0700241C07002424070024EE
:10A65000240700242C0700242C070024340700249E
:10A66000340700243C0700243C070024440700244E
:10A67000440700244C0700244C07002454070024FE
:10A68000540700245C0700245C07002464070024AE
:10A69000640700246C0700246C070024740700245E
:10A6A000740700247C0700247C070024840700240E
:10A6B000840700248C0700248C07002494070024BE
:10A6C000940700249C0700249C070024A40700246E
:10A6D000A4070024AC070024AC070024B40700241E
:10A6E000B4070024BC070024BC070024C4070024CE
:10A6F000C4070024CC070024CC070024D40700247E
:10A70000D4070024DC070024DC070024E40700242D
:10A71000E4070024EC070024EC070024F4070024DD
:10A72000F4070024FC070024FC070024040800248C
:10A73000040800240C0800240C0800241408002439
:10A74000140800241C0800241C08002424080024E9
:10A75000240800242C0800242C0800243408002499
:10A76000340800243C0800243C0800244408002449
:10A77000440800244C0800244C08002454080024F9
:10A78000540800245C0800245C08002464080024A9
:10A79000640800246C0800246C0800247408002459
:10A7A000740800247C0800247C0800248408002409
:10A7B000840800248C0800248C08002494080024B9
:10A7C000940800249C0800249C080024A408002469
:10A7D000A4080024AC080024AC080024B408002419
:10A7E000B4080024BC080024BC080024C4080024C9
:10A7F000C4080024CC080024CC080024D408002479
:10A80000D4080024DC080024DC080024E408002428
:10A81000E4080024EC080024EC080024F4080024D8
:10A82000F4080024FC080024FC0800240409002487
:10A83000040900240C0900240C0900241409002434
:10A84000140900241C0900241C09002424090024E4
:0CA8500024090024FFFFFFFF00000200AD
:04000005080013CD0F
:00000001FF
